:100000000C9426030C946D030C946D030C946D03F7
:100010000C946D030C946D030C946D030C946D03A0
:100020000C946D030C946D030C94B8310C948C32C9
:100030000C94542C0C946D030C946D030C946D0370
:100040000C946D030C946D030C946D030C946D0370
:100050000C946D030C94AB2C0C946D030C946D03F9
:100060000C946D030C946D030C946D030C946D0350
:100070000C946D030C946D030C946D030C946D0340
:100080000C946D030C946D030C946D030C946D0330
:100090000C946D030C946D030C946D030C946D0320
:1000A0000C946D030C946D030C946D030103E1013A
:1000B00003E2000102E10102E2002B0014001A0039
:1000C0000800150017001C0018000C001200130097
:1000D000294104001600070009000A000B000D006A
:1000E0000E000F003441E1001D001B000600190046
:1000F000050011001000380000000251E00002511C
:10010000E300000000002C00E600E50003530000BF
:100110002A0000000000000000002A2B2800000038
:1001200000000000000000000000000000290000A6
:1001300000002C1E3420212224342627252E362D83
:100140003738271E1F202122232425263333362E1D
:1001500037381F0405060708090A0B0C0D0E0F108F
:100160001112131415161718191A1B1C1D2F3130D4
:10017000232D350405060708090A0B0C0D0E0F1078
:100180001112131415161718191A1B1C1D2F3130B4
:10019000354C0000000000000000000000000000DE
:1001A000000000000000000000000000000000004F
:1001B0000000000000007E0F00D4FFFFFFC700001A
:1001C0000078FD377A585A000004E6D6B44602009B
:1001D000210116000000742FE5A3E0058001D15D28
:1001E000003D8889C65436C3174FE4DF231EE1A6BD
:1001F000EDA9C348EB9A8A89C88899C57D1B16A6C4
:10020000699ED92B8DD015F22F3120F2790D50AF88
:10021000978E750BF3DC9F72A108B0706EA698BA2A
:1002200046397C76929EDD347999D6B2312A817C2A
:10023000D5CE198326CB837BFAA2035E8062FA4077
:100240002DCA76CF12F2B968E12B92040DE316CFD6
:1002500042224805A88AA22D20FCFA6E5609A397CF
:100260000B5317B367B2ECD2E08ED961F510305161
:1002700003A7AE2D4332F621DA5352AE4C8D1B6FDD
:100280005B2051ADA29736454EAA2DF26A3E2EC094
:10029000B727286BB004B4F54E736915DD036210FF
:1002A0003CEF4CA5BC8B8894A65510E04D6268C10C
:1002B00093BAED0BD91D37E1C21548B792EDC3CD06
:1002C00080F2ADF8990A5BC1EBE9F8D9A654D5479D
:1002D000B14D48A34AA16D31A4FE1B85055482850A
:1002E00043D66DDF6D2C89C8E6A65264CE4D40FB27
:1002F000BAF24AFA256F7B9FB54B1CB69347A627E7
:10030000C17B81C1B5E55B2B39B2536B5ECB03EB8F
:1003100041E5C8BBFAABB301CC600A6FF215AE463B
:10032000855B1724049FE1586184DD755A906161F3
:10033000E680F5810CBFC410862632F6AE4D605AB9
:100340006773A2FF1637C1DDD8A08166551288AA4F
:100350003C6CD2C727643923F6F0721C3CD0BA1526
:100360005217A764DC2951FE31845D94CCB9517FCA
:100370003FDCD924E51368807BB99358C5B51D339C
:10038000DF434DD50B43CC7361408CCE441AFAA6A3
:10039000AB79BB1616EE14DDE3C7AED7540D15E4EA
:1003A000EB9E843A961A2E0DD6B3336C432CE4FBA5
:1003B00013870000000086A91B647F0D4BEA000133
:1003C000ED03810B0000EE989F77B1C467FB02003C
:1003D00000000004595A01000100770400000200E7
:1003E0000200730400000300010078040000040010
:1003F00002005D044B2105000100790400000600A5
:1004000002005F04000007000200750400000800FD
:1004100001007A04000009000200610426210A009C
:100420000200630426210B000200650426210C0053
:100430000200670426210D000200690426210E0037
:1004400002006B0426210F0002006D04262110001B
:1004500002006F04262111000200710426211200FF
:1004600002007B040000130002007D0400001C0356
:100470007600690061006C003A00660036003400C6
:100480006300320062003300630000000A0347008B
:100490006F006F006E0000002203540068006500CA
:1004A000560061006E0020004B006500790062007C
:1004B0006F0061007200640073000000040309040F
:1004C00009025B00030100A03209040000010301DE
:1004D00001000921110100012240000705810308E4
:1004E000000A0904010002030000000921110100B3
:1004F00001222200070582032000010705030320D3
:10050000000109040200010300000009211101009B
:100510000122BC000705840320000A12010002002A
:10052000000008AEFE47880100010203010660FFDB
:100530000961A1010962150026FF00952075088157
:10054000020963150026FF00952075089102C00579
:10055000010902A10185020901A10005091901296A
:100560000515002501950575018102950175038129
:10057000010501093009311581257F950275088132
:100580000609381581257F950175088106050C0A35
:1005900038021581257F950175088106C0C00501C7
:1005A0000980A101850319012AB700150126B700AA
:1005B000950175108100C0050C0901A10185041980
:1005C000012AA002150126A002950175108100C024
:1005D00005010906A1018505050719E029E71500B0
:1005E00025019508750181020507190029EF1500FD
:1005F000250195F075018102050819012905950568
:1006000075019102950175039101C005010906A1CB
:1006100001050719E029E7150025019508750181F5
:10062000029501750881010507190029FF150026AB
:10063000FF00950675088100050819012905950533
:1006400075019102950175039101C00011241FBE2F
:10065000CFEFDAE0DEBFCDBF04B603FE27C0809146
:10066000900490919104A0919204B09193048730EA
:10067000904BA740B04BD1F410929004109291048B
:10068000109292041092930414BE84B7877F84BFA3
:100690000FB6F894A89580916000886180936000FF
:1006A000109260000FBEE0E0F8E3099511E0A0E0D1
:1006B000B1E0ECE3FAE602C005900D92A63AB1076C
:1006C000D9F724E0A6EAB1E001C01D92A039B20733
:1006D000E1F70E94A9160C94E6340C940000CF9325
:1006E000DF93A1E3B1E045E351E0C1E0D0E08D91BB
:1006F000E82FE295EF70F0E061A18F709E0101C0DC
:10070000220F8A95EAF7922F9095962391A382A1C2
:10071000822B82A34A175B0751F7A6E2B1E041E3BF
:1007200051E0C1E0D0E08D91E82FE295EF70F0E06C
:1007300061A18F709E0101C0220F8A95EAF7922F66
:100740009095962391A382A1822B82A34A175B07DF
:1007500051F7DF91CF9108956F927F928F929F9280
:10076000AF92BF92CF92DF92EF92FF920F931F93BF
:10077000CF93DF9321E3C22E21E0D22E8C015C01C6
:1007800088E0A80EB11C712C88248394912CF6016A
:1007900081916F01C82FC295CF70D0E099A18F7061
:1007A000740101C0EE0C8A95EAF7892F8E2989A37E
:1007B0008AA16E2C609486218AA30E943616E6E2F6
:1007C000F1E050E040E030E020E06191A62FA295FA
:1007D000AF70B0E090968C9190E06F7002C09595EC
:1007E00087956A95E2F780FD34C0C401042E02C0EB
:1007F000880F991F0A94E2F7282B392B4F5F5F4F20
:100800004B30510511F789A1682269A28AA1E82A13
:10081000EAA2F8018081918128173907E9F0318334
:10082000208381E0782A0E5F1F4F0A151B0509F00F
:10083000AECF872DDF91CF911F910F91FF90EF9059
:10084000DF90CF90BF90AF909F908F907F906F90F0
:10085000089590E080E0D0CF80E0E4CF0C942A1699
:100860000C942B160C9436040C94FF06CF93FB01CA
:10087000C281CC2359F082369D4529F483EB90E068
:100880000E94FC06C0E08C2FCF91089582369D45D2
:1008900029F48CEA90E00E94FC06F5CFC1E0F3CF8A
:1008A0009C013A9521153F4150F5FC01EE27F1706E
:1008B000BC0166277270AC01442754709C0122274A
:1008C000387094FF0EC080E1EF2B09F480E0672BB5
:1008D00009F08062452B09F08064232B89F0806841
:1008E000089581E0EF2B09F480E0672B09F0826026
:1008F000452B09F08460232B19F08860089580E06F
:100900000895CF93DF93EC010E9450049E01205E76
:1009100031092830310510F0209739F40E9424085D
:100920008C2FDF91CF910C9484070E943208F8CF6E
:10093000CF93DF93EC010E94D207CE010E945004B6
:100940009E01205E31092830310510F0CD2B21F4B5
:10095000DF91CF910C942B08DF91CF910C94390843
:1009600081E0089508950C94B2041F93CF93DF9310
:1009700000D000D00F92CDB7DEB749835A836B8386
:100980003091A80189819A8131111DC06623B9F087
:100990002223A9F00E94300C182F682F89819A8198
:1009A0000E94D30B69817A81812F0F900F900F9055
:1009B0000F900F90DF91CF911F910C940D200E940A
:1009C000030C182FEFCF0E94300C69817A81EDCF94
:1009D000FC01262F86819781009739F4408151814F
:1009E0006281738184810C94B5040895CF93DF9361
:1009F000EC0161E00E94E804BE01DF91CF910C940C
:100A00008D26CF93DF93EC0160E00E94E804BE01E5
:100A1000DF91CF910C94B304E1E0F0E0DF0102C07C
:100A2000AA0FBB1F6A95E2F7BD01DF0102C0AA0F42
:100A3000BB1F4A95E2F76A2B01C0EE0F2A95EAF731
:100A4000962F9823961302C08E2B0895E0958E233F
:100A50000895242F462F682F8091BD010E940C0518
:100A60000C94900B0E9410160E9404070C942E0404
:100A70000E9464290E9449260E94222A0C94300474
:100A800008950E9456080E9440052FEF84E39CE0E1
:100A9000215080409040E1F700C000000C94CF2C22
:100AA0000F931F93CF93DF93EC018B010E94C22819
:100AB000B801CE010E94C319882309F448C0B801C7
:100AC000CE010E943204882309F441C0B801CE014E
:100AD0000E940A298823D9F1B801CE010E94852AF3
:100AE0008823A9F1B801CE010E940723882379F158
:100AF000B801CE010E945923882349F1B801CE01E3
:100B00000E947C24882319F1F8018281882361F0F6
:100B1000CA35FDE5DF0721F170F4C115ECE5DE070C
:100B2000A1F0CE3DDC45C9F0C801DF91CF911F9106
:100B30000F910C94B004CB358DE5D807A1F0CC35DE
:100B4000DD4591F70E944A11EFCF0E94410580E0F8
:100B5000DF91CF911F910F9108950E94FF12F7CF5F
:100B60000E945311E1CF0E945611DECFCF93DF9345
:100B7000EC0161E00E94E804BE01DF91CF910C948A
:100B80005005DF92EF92FF920F931F93CF93DF9365
:100B9000E82FF0E0EE5EFE4FD490282F26952695A4
:100BA000269530E0F901EE54FE4F0491877010E075
:100BB000082E02C0159507950A94E2F701701127D7
:100BC000F901EE55FE4FE490F12C082E02C0F59489
:100BD000E7940A94E2F791E0E922FF24F901EE5646
:100BE000FE4FC491D0E002C0D595C7958A95E2F733
:100BF000C170DD270115110519F081EE0E948407EF
:100C0000E114F10419F086EE0E9484078D2D0E94F4
:100C10001808EF2819F086EE0E94D207012B19F070
:100C200081EE0E94D207CD2B51F08CE2DF91CF9163
:100C30001F910F91FF90EF90DF900C941808DF91B7
:100C4000CF911F910F91FF90EF90DF900895EF9259
:100C5000FF920F931F93CF93DF93EC01162F0AE0BF
:100C60008881882309F454C0813009F04EC08981FD
:100C7000813099F47E0122E0E20EF11C8A810E940B
:100C80001808E7012196812F815050F3EFE9FFE02A
:100C90003197F1F700C00000F7CF823041F47E01B8
:100CA00082E0E80EF11C8A810E948407EACF83303B
:100CB00041F47E01E2E0EE0EF11C8A810E94D2072F
:100CC000E0CF843011F02196DDCF2A81229690E08A
:100CD00080E0AE014F5F5F4F2053330B2A30310568
:100CE00048F0019778F2EFE9FFE03197F1F700C0A3
:100CF0000000F7CF089FB001099F700D1124C901B2
:100D0000860F971F2981EA01E4CF0E94C105BACF5F
:100D1000DF91CF911F910F91FF90EF90089560E0C8
:100D20000C942706EF92FF920F931F93CF93DF93BC
:100D30008C01F62E8AE0E82EF8018491882309F4CC
:100D400054C0813009F04DC0E8012196FE01849124
:100D5000813091F42196FE0184910E9418088E0141
:100D60000F5F1F4F8F2D815038F3EFE9FFE0319770
:100D7000F1F700C00000F7CF823039F4E801229685
:100D8000FE0184910E948407EACF833039F4E801A0
:100D90002296FE0184910E94D207E1CF8430F9F6B9
:100DA000E8012296FE01249190E080E0FE01319658
:100DB0002053330B2A30310548F0019780F2EFE9D8
:100DC000FFE03197F1F700C00000F7CFE89EA001E7
:100DD000E99E500D1124C901840F951F2491EF0144
:100DE000E5CF0E94C105E801BACFDF91CF911F91F5
:100DF0000F91FF90EF90089560E00C949206089593
:100E000081E008950C9400070895CF93C82F0E94A5
:100E100034048C2FCF910C940207019708F40895A5
:100E2000EFE9FFE03197F1F700C00000F6CFCF9374
:100E3000DF93CDB7DEB72D970FB6F894DEBF0FBEA8
:100E4000CDBF49875A876B877C878D878C859D8529
:100E5000892B29F0CA0189238F3F09F046C08B8571
:100E600081110E947C111D821E821F82188685E0DE
:100E7000FE013996DE01119601900D928A95E1F7F7
:100E800080915F0490916004892B61F00E9417119A
:100E9000882319F082E00E9439120E94F310811118
:100EA0000E94C3118C819D81892B99F429813A81FB
:100EB0004B815C816D817E818F8198850E943C1081
:100EC0002D960FB6F894DEBF0FBECDBFDF91CF9148
:100ED000089589819A8189238F3F41F3CE0101963C
:100EE0000E94F6048111E2CFEBCF8091A90190918D
:100EF000AA0101969093AA018093A901B0CFFC01A9
:100F0000808191810C945D0CCF93C82F882309F4C4
:100F100047C08CEF8C0F813AA0F46C2F80910001B8
:100F2000909101010E94A02B882329F08C2F0E9410
:100F3000E3100E94D1118C2F0E94DC10CF910C94F1
:100F4000D11180E28C0F883048F4C77081E001C075
:100F5000880FCA95EAF70E945C11F0CFEBE5EC0F21
:100F6000E33040F4F0E0ED59FE4F808190E0CF9106
:100F70000C94602BE8E5EC0FE73150F4F0E0EE0F55
:100F8000FF1FEB5CFE4F80819181CF910C94762BFB
:100F9000C03F30F08C2F0E944C17CF910C94371823
:100FA000CF910895882361F19CEF980F913A20F436
:100FB0000E94E3100C94D11190E2980F983050F4F5
:100FC000877091E001C0990F8A95EAF7892F0E94F6
:100FD0006211F0CF9BE5980F933020F490E080E011
:100FE0000C94602B98E5980F973120F490E080E006
:100FF0000C94762B803F20F00E94B4170C94371885
:1010000008951F93CF93DF93182FEB010E9484075D
:10101000209731F4812FDF91CF911F910C94D2074B
:101020008FE99FE00197F1F700C000002197F0CF12
:1010300060917D0470917E04893321F060917B047E
:1010400070917C040C940108882321F00E945C11AB
:101050000C94D1110895882321F00E9462110C9400
:10106000D1110895882321F00E946F110C94D111A1
:101070000895882321F00E9475110C94D1110895D0
:1010800090E080E00E94602B90E080E00E94762B50
:101090000E947C110E948C110E94D1110E945E1945
:1010A0000C9437180E94EA100C9440080E946911B1
:1010B0000C945208E92FE295EF70E250EE3070F494
:1010C000F0E0E851FB4C0C946634803F19F020F4BA
:1010D000883E20F481E00895843FE1F380E00895A4
:1010E000883EC0F3813FD1F7F5CF93FB882780F985
:1010F0000895FC0186819781009721F00E940514D4
:101100000C945A08808191810E945D0CF9CFBF92A6
:10111000CF92DF92EF92FF920F931F93CF93DF93C3
:101120007C01EB01FC010281158112951F700E9468
:101130003111C82E8823A1F0C02E002389F08D2FF5
:10114000807F803429F080E28C0FC12C883040F001
:1011500082E00E9439120E94311191E0C82EC92606
:10116000BD2EB2942FE0B222EB2DF0E0EA50FB4C02
:101170000C946634FD2FFF70DF2E8D2F807F19F0C9
:10118000D29490EFD9220023A9F0DD2059F080E21B
:101190008C0F883010F0C11109C08D2D0E945C1198
:1011A0000E94D1118C2F0E94840714C08D2D0E94A3
:1011B0006F11F6CF8C2F0E94D207DD2059F080E20C
:1011C0008C0F883010F0C11134C08D2D0E94621137
:1011D0000E94D111EB2DE850FF0B349720F40E94B0
:1011E0002C2B0E940507CE010E945A088111E6C1EE
:1011F0001092AA011092A901CC2009F400C20E9409
:10120000131180FDFCC1F70112820E940D110E9492
:10121000A10BC7010E94270B0E940D11DF91CF91F6
:101220001F910F91FF90EF90DF90CF90BF900C94A3
:10123000AC0B8D2D0E947511CBCF2D2F2F70D22E80
:101240008D2F807F803219F0D29480EFD822CC236A
:10125000E9F0C13009F455C0002309F45CC0112342
:1012600091F120E0F7014081518162817381848195
:101270000E94B504B7010E946622811193CFF70145
:10128000858180FF8FCF8F7085831DC00023E9F09B
:10129000111106C00E948F118D290E9424089ACF37
:1012A000113031F40E948F118D290E94AB1192CF21
:1012B00080917904823070F38113ECCF0E94C311C6
:1012C0008D2D0E9495118D2DE8CF111106C00E9421
:1012D000C3118D2D0E942B087DCF80917904113090
:1012E00059F4823008F476CF0E9459118D2109F407
:1012F00071CF0E949E11EBCF823048F31813E7CFD5
:1013000069CF002321F0163008F064CFDCCF153010
:1013100008F060CFDECF1123E1F280917D0490913F
:101320007E04C93321F080917B0490917C040E945B
:101330000D078C2F0E94D2074DCF8D2F8695869555
:10134000837061F0813009F045CFCE0193700111B7
:1013500002C090E080E00E94762B3CCFCE019370DB
:10136000011102C090E080E00E94602B33CF8C2FEF
:10137000002339F00E944C170E9437180E9437183A
:1013800029CF0E94B417FACF8D2F837081F50111F8
:1013900021CF4C2F429546954770440F440F8C2F18
:1013A0008F70042E01C0880F0A94EAF72C2F207149
:1013B000C4FF07C02FE030E001C0220F4A95EAF7D2
:1013C00020959D2F969596959370822B923049F09B
:1013D00058F4913019F00E94820BFCCE0E947D0BD4
:1013E000F9CE0E94870BF6CE0E947B0BF3CE86953A
:1013F000002311F08D2F8170882309F4EBCE4C2F40
:10140000429546954770440F440F8C2F8F70042EE1
:1014100001C0880F0A94EAF72C2F2071C4FF07C07F
:101420002FE030E001C0220F4A95EAF720959D2F6A
:10143000969596959370822B923049F058F491309E
:1014400019F00E94C80BC6CE0E94C30BC3CE0E94E7
:10145000CD0BC0CE0E94900BBDCEFD2FFF70DF2EB6
:10146000002329F08F2F0E94A10B8C2F16CF8C2FD9
:101470000E942B088D2D0E94AC0BACCEC23F09F40C
:101480003FC060F4C03F31F1C13F91F1002309F446
:1014900080C0111187CE8D2F8F712FC0C33FA9F14E
:1014A000C43FA1F780917904823008F45BC0002327
:1014B00009F444C00E94F0100E9462110E941311AE
:1014C000843069F50E9430128D2F8F710E94AC0B11
:1014D000C12C80CE002341F0153008F07BCE8D2F3B
:1014E0008F710E94B80B76CE163008F073CEF7CF0E
:1014F0008D2F8F71002309F4BECF0E94A10B6ACEFD
:101500008D2F8F710023C9F3B6CF002329F08D2FC3
:101510008F710E94990B5ECE0E94960B5BCE8091DC
:1015200079041817A8F62D2F2F71D22E822F0E9422
:10153000A10B63E08D2D0E941412CACF0E94F010FF
:101540000E945C1180917904181740F00E943012BB
:101550000E949E1164E08D2F8F71EDCF81E00E947B
:101560003912B6CF002359F03D2F3F71D32E832F70
:101570000E94A10B63E08D2D0E9414122BCE81E0FE
:101580000E943912123008F425CE82E00E943912EE
:1015900021CE1111C2CE8D2F8F716DCF4D2F4F7077
:1015A0006C2FC7010E94F9130E948B0C13CE4D2F94
:1015B0004F706C2FC7010E94FC130CCE002319F052
:1015C000111116CE19CE111113CE20E0F701408172
:1015D00051816281738184810E94B504B7010E94A8
:1015E0007122882309F404CE8091A9019091AA0167
:1015F000029709F0FDCD8C2F0E941808F9CDDF91DC
:10160000CF911F910F91FF90EF90DF90CF90BF90FF
:1016100008950F931F93CF93DF93EC018E819F81E9
:10162000009779F00E9405148C010E94D20B0E9451
:101630007A0BB801CE01DF91CF911F910F910C94DD
:101640008708688179818A810E94670CEDCFCF93EA
:10165000DF93EC018B819C81892B29F08881998112
:1016600089238F3F59F4DF91CF910895CE010E94D5
:10167000090BCE01DF91CF910C940105CE010E94A0
:10168000B6058111F3CF0E943111882361F38A815D
:10169000882349F382E0DF91CF910C943912CF93E4
:1016A000DF9300D000D00F92CDB7DEB70F900F9030
:1016B0000F900F900F90DF91CF910895CF93DF930C
:1016C000CDB7DEB728970FB6F894DEBF0FBECDBFFB
:1016D00028960FB6F894DEBF0FBECDBFDF91CF9135
:1016E000089508950C94710B0E94720B8093BE01B3
:1016F0000C94400808950C94740B9091BE01892BB2
:101700000C94740B9091BE0189230C94740B9091EE
:10171000BE0189270C94740B0C94710B0C948C0BE8
:101720000E948E0B8093BD010C94400880E00C94C5
:10173000900B91E001C0990F8A95EAF7892F0C94DC
:10174000900B21E030E001C0220F8A95EAF78091EA
:10175000BD01822B0C94900B21E030E001C0220FE0
:101760008A95EAF720958091BD0182230C94900B15
:1017700021E030E001C0220F8A95EAF78091BD0197
:1017800082270C94900B9091BD01892B0C94900BA7
:101790009091BD0189230C94900B9091BD018927F4
:1017A0000C94900B08959E3F69F1E82F2BE0929FD7
:1017B000E00D11248E2F877041E001C0440F8A95FF
:1017C000EAF7E695E695E69583E0E89FF0011124B7
:1017D000E555FE4F30E020E070E05191DF011197B8
:1017E000CB01022E02C0969587950A94E2F781708C
:1017F00081958527842385278C932F5F3F4F233046
:10180000310559F708959E3F49F1E82F2BE0929F4B
:10181000E00D11249E2F9770E695E695E69583E0FE
:10182000E89FF0011124E555FE4F50E040E080E0D4
:10183000219130E0092E02C0369527950A94E2F7EF
:1018400021703327042E01C0220F0A94EAF7822B5D
:101850004F5F5F4F4330510559F7089580E0089579
:10186000CF92DF92FF920F931F93CF93DF936C0180
:101870000091BD018091BE01082BC7E0D0E010E0CF
:10188000FC2EC8010C2E02C0959587950A94E2F7AC
:1018900080FD0CC02197A0F7F12C8F2DDF91CF9107
:1018A0001F910F91FF90DF90CF900895B6018C2F7C
:1018B0000E941815019771F3F0CFCF93DF93EC01DD
:1018C0000E94300CBE01DF91CF910C9418151F932C
:1018D000CF93DF93EB019091A801992331F0CB01D5
:1018E000DF91CF911F910C945D0C882379F0CB018F
:1018F0000E94300C182F682FCE010E94D30BBE011E
:10190000812FDF91CF911F910C941815CB010E946C
:10191000030C182FF4CFEF92FF920F931F93CF93E6
:10192000DF938C01892B81F0F12CEE24E394E80104
:101930002196F8018491843770F4843008F05FC0F8
:101940008130B1F08230A1F1DF91CF911F910F91E1
:10195000FF90EF900895853709F44CC008F43DC01E
:101960009CE7980F903780F78F770E94D20749C085
:101970000E5F1F4FFE01849190E2980F983060F443
:101980008770FE2D01C0FF0F8A95EAF78F2F0E9406
:101990007F110E94D11102C00E9484078F2D8150B7
:1019A00030F2EFE9FFE03197F1F700C00000F7CF28
:1019B0000E5F1F4FFE01849190E2980F983050F413
:1019C0008770FE2D01C0FF0F8A95EAF78F2F0E94C6
:1019D0008511DFCF0E94D207E1CF0E5F1F4FFE01BE
:1019E000C491C150D8F28FE99FE00197F1F700C090
:1019F0000000F7CF0E5F1F4FFE01F490CFCF0E9483
:101A000084078E01CBCFCF93DF93C091BF0180912C
:101A1000C0018C1303C0DF91CF910895D0E0FE0187
:101A200083E0EE0FFF1F8A95E1F7EF53FE4F208111
:101A300031814281538164817581868197810E94C1
:101A40005E0B2196C770E3CF209101023091020214
:101A500040910302509104026091050270910602C8
:101A600080910702909108020C945E0B2091BF01B7
:101A70009091C001291302C080E0089530E0F9017F
:101A800053E0EE0FFF1F5A95E1F7EF53FE4F5181E0
:101A9000561306C05081581303C05281541304C01A
:101AA0002F5F3F4F2770E6CF81E00895EF92FF92BE
:101AB0000F931F93CF93DF9380910602807F31F4C1
:101AC00080910302C091BF01811119C0DF91CF91B4
:101AD0001F910F91FF90EF90089520910402309193
:101AE0000502D0E02115310541F08091010290916D
:101AF0000202482F49234F3F39F42196C770809145
:101B0000C0018C13EACFE2CF8E0143E0000F111F1A
:101B10004A95E1F7F801EF53FE4F41814913EDCFAC
:101B200090819813EACF82818111E7CFE380F4801E
:101B3000E21AF30A60E081E092E00E94E80461E0CA
:101B400072E00E945D22E816F906B8F6809106025E
:101B50008F70806180930602F801EA53FE4F808106
:101B60008F708061808381E092E00E94270BDF917B
:101B7000CF911F910F91FF90EF900C94030D6F92F6
:101B80007F928F929F92AF92BF92CF92DF92EF920D
:101B9000FF920F931F93CF93DF93CDB7DEB7659777
:101BA0000FB6F894DEBF0FBECDBF8C0185E0F80103
:101BB000DE01519601900D928A95E1F7D8011296B7
:101BC000FC90129781E0882E82E0982E20910402EA
:101BD000309105022115310541F08091010290916B
:101BE000020289238F3F09F0E9C1F11010C1C80139
:101BF0000E94270B82C060E081E092E00E94E8042E
:101C0000B8010E946222811116C2CD2829F0872DC9
:101C100086218F3F09F011C180E0B82FB170CB2E23
:101C200080FF29C04F2D672D862D0E94360DD82E9E
:101C3000811121C0698A7A8A89899A890E945D0CFA
:101C4000292F22952F70223050F0243078F49F7085
:101C500051F0F8019581907F31F4ED2C1AC19F70FD
:101C600011F08823D1F3805E8830B8F3C8010E9458
:101C7000270BDC2CF2CFFF2009F40BC18091060268
:101C8000816080930602E12C04C1892B49F0809188
:101C9000010290910202282F29232F3F09F00FC142
:101CA000C8010E947908882309F4A1CFFF2009F414
:101CB0009ECF809106028032A0F0209101023091E7
:101CC00002023A8729871B86DD86CC868E87809123
:101CD000070290910802988B8F87CE0109960E9487
:101CE000270B88E0F801A1E0B2E001900D928A95FF
:101CF000E1F70E94560D0E94240DEE24E394C9C022
:101D0000211112C07C2DDD8ACC8AA3016F2D8D8913
:101D10000E944F0B81E092E00E94270B88E0F401C3
:101D200011928A95E9F7A5C180910402909105026C
:101D3000892B49F08091010290910202282F2923DA
:101D40002F3F09F0E4C0C8010E947908882309F4F4
:101D50004ECFFF2009F44BCF80910602803208F26B
:101D600020910102309102023A8329831B82DD8295
:101D7000CC828E83809107029091080298878F838E
:101D8000CE010196ACCF60E081E092E00E94E804D1
:101D900061E072E00E945D22A816B90650F5EF2CB2
:101DA000FF2009F424CF8091040290910502892B31
:101DB00049F08091010290910202282F29232F3FA0
:101DC00009F0CBC0C8010E94790881118ACF8091A7
:101DD0000602816080930602C8010E94270B59C049
:101DE00088E0F801A1E0B2E001900D928A95E1F758
:101DF00050C07C2DDD8ACC8AA3016F2D8D890E9475
:101E00004F0B88E0F40111928A95E9F77DC0C80173
:101E10000E947908E82E882309F4E9CE88E0F801C9
:101E2000A1E0B2E001900D928A95E1F781E092E0A5
:101E30000E947F070E94560D67C081E08F25EDCE7E
:101E400081E08F2501C1D80111962C912913E7C09B
:101E5000F80190819813E3C02091070230910802A5
:101E6000868197812817390709F0D9C0F110D7C0AA
:101E7000809106028F708061809306020E94240D7B
:101E800081E092E00E94270B80910602D80115960E
:101E90008C938E2D65960FB6F894DEBF0FBECDBF26
:101EA000DF91CF911F910F91FF90EF90DF90CF9036
:101EB000BF90AF909F908F907F906F900895F801A2
:101EC00021812913EDCED8019C919813E9CE209160
:101ED00007023091080216968D919C91179728174A
:101EE000390709F0DDCE80910602F110D9CE1596A2
:101EF0008C93C8010E94270B88E0F801A1E0B2E0B2
:101F000001900D928A95E1F70E94240DC2CFD8016D
:101F100011962C91291317CFD8019C91981313CFA8
:101F2000209107023091080216968D919C91179787
:101F30002817390709F007CFF11005CF8091060265
:101F400015968C93C8010E94270BE1E0F2E088E02F
:101F5000DF011D928A95E9F79CCFF80121812913B1
:101F600031CFF801908198132DCF20910702309145
:101F70000802868197812817390709F023CF60E08E
:101F800081E092E00E94E804B8010E946B22811176
:101F900027CF8091060280FD23CF982F907F09F4F0
:101FA0001FCFD80115968C931597903F09F4A1CFB8
:101FB000982F907F905F8F70892B99CF6C9011969E
:101FC0007C9011971396CD90DC90E090030256011F
:101FD000A21AB30AEE2009F4D6CE60E081E092E0C6
:101FE0000E94E80461E072E00E945D2220910602F6
:101FF000207FA816B90608F083CE80910402909144
:102000000502211142CEEF2C892B49F0809101026B
:1020100090910202282F29232F3F09F014CF60E06E
:1020200081E092E00E94E804B8010E945D22843FB2
:10203000914008F4E0CDC114D10429F0872D862108
:102040008F3F09F0FDCE80E080FFDFCD4F2D672D63
:10205000862D0E94360D882309F4D7CD81E092E0C9
:102060000E94270B88E0E1E0F2E0DF011D928A95F3
:10207000E9F70E94240D07CECF93DF93CDB7DEB7EB
:1020800060970FB6F894DEBF0FBECDBF29873A87A1
:102090004B875C876D877E878F87988BCE010996EB
:1020A0000E94BF0D8823D1F08C859D85892B39F046
:1020B00029853A85822F83238F3F09F074C0809150
:1020C000BF019091C001891348C060960FB6F89483
:1020D000DEBF0FBECDBFDF91CF91089588E0FE0136
:1020E0003996DE01119601900D928A95E1F78C8563
:1020F0009D85892B21F389859A8589238F3FF9F264
:10210000A091C001B0E0CD01019687709927209180
:10211000BF012817190671F40E9456081092C001D9
:102120001092BF0188E0E1E0F2E0DF011D928A95A4
:10213000E9F7C5CF93E0AA0FBB1F9A95E1F7AF531C
:10214000BE4F98E0FE01319601900D929A95E1F70D
:102150008093C0010E94030DB2CFB8E08B9FC001F5
:1021600011248F539E4F0E94BF0D882309F4ADCFD9
:10217000E091BF0128E0E29FF0011124EF53FE4FF0
:10218000208131814281538164817581868197816B
:102190000E945E0B8091BF0190E0019687709927A5
:1021A0008093BF018CCF4B855C856D857E858F8547
:1021B00098890E945E0B83CF682F809100019091D7
:1021C00001010C94202C682F809100019091010155
:1021D0000C942B2C80910001909101010C94362CD1
:1021E00080910E02089580915F0490916004892B84
:1021F00089F00E94842C20910C0230910D02AC01D8
:10220000421B530B81E020915F0430916004421720
:10221000530708F480E08170089580910B02859542
:1022200085958595089580910B02877008950E9489
:10223000842C2091090230910A02821B930B209179
:102240005F04309160048217930748F080910B027D
:1022500082FB882780F991E089278170089580E0CA
:10226000FCCF90910B02977081E009F480E0089513
:102270009091120392FB222720F9281751F080FB3E
:1022800092F99093120380911103909112030C9490
:102290007C1208958091120382FB882780F991E0D7
:1022A00089270C94381181E00C94381180E00C944B
:1022B000381180913202089590913202892B8093D7
:1022C00032020895809590913202982390933202C1
:1022D00008951092320208958091310208959091EC
:1022E0003102892B809331020895809590913102BB
:1022F000982390933102089510923102089590919D
:102300003002892B8093300208958095909130029D
:10231000982390933002089510923002089580918E
:102320000F02089508950C94921190910E0298173F
:1023300021F080930E020C949311089580910E0267
:10234000882329F010920E0280E00C9493110895D6
:1023500008950C94A811CF93C82F8091120382FD89
:1023600010C080910F028C1761F00E94842C909312
:102370000D0280930C02C0930F028C2FCF910C940E
:10238000A911CF91089580910F02882349F01092EE
:102390000F0210920D0210920C0280E00C94A91111
:1023A0000895E0910001F091010180913202808353
:1023B000E0910001F0910101808190913102892B1F
:1023C0008083E0910001F0910101808190913002C1
:1023D000892B808380910F028823E9F080915F042C
:1023E00090916004892B29F00E94F31081110E94C2
:1023F000C311E0910001F0910101808190910F02E1
:10240000892B808380910001909101010E948C2B87
:1024100081110E94C31180910001909101010C94DF
:10242000382B08950C9411129091120392FD16C04E
:1024300098E0899F90011124622B60930B020E9407
:10244000A10B0E94842C90930A0280930902809130
:102450000B028595859585950C9412120C94A10B11
:1024600010920B0210920A021092090280E00C9462
:10247000121290910B028095892380930B02282FD2
:10248000277039F4282F082E000C330B92171306EF
:1024900021F49091120392FF07C08595859585954B
:1024A0000E94AC0B0C94301208956FEF7FEF90E018
:1024B00080E00C94C83490E080E00E94A4348A3E0E
:1024C0009E4F11F40C946C1980E0089582E090E026
:1024D0000C949C3483E090E00C949C34CF9384E083
:1024E00090E00E949C34C82F82E290E00E949C34CD
:1024F000982F8C2FCF910895CF93C92F682F84E008
:1025000090E00E94AA346C2F82E290E0CF910C946C
:10251000AA34AB01BC018FE090E00C94BC34AB0159
:10252000BC0183E190E00C94BC3460E070E0CB012E
:102530000C948F1260E070E0CB010E9489120C9421
:1025400095126AEE7EEF90E080E00E94C83460E071
:1025500082E090E00E94AA3460E083E090E00E9474
:10256000AA341092BE0160E084E090E00E94AA3498
:1025700060E082E290E00E94AA3460E085E090E0B2
:102580000E94AA3460E086E090E00E94AA346FEFD7
:1025900087E090E00E94AA3440E050E0BA0188E071
:1025A00090E00E94BC3460E08DE090E00E94AA348C
:1025B00040E050E0BA0188E190E00E94BC3460E065
:1025C00087E190E00E94AA3440E050E0BA018CE13B
:1025D00090E00E94BC3470E060E080E290E00E94F5
:1025E000C83440E050E0BA0188E190E00E94BC3479
:1025F00080E00E9485190E94AB190C949A120C94E9
:10260000A112682F8EE090E00C94AA340E94902CC6
:102610006093400270934102809342029093430280
:1026200060933C0270933D0280933E0290933F0280
:10263000089585B7806885BF85B7806885BF089590
:10264000089508950C94201308950C9424130E9467
:10265000191386EF95E10E94F32C0E942A1D0E9417
:102660006D210E9421130C94221381E008950C9493
:102670003513089508950E9439130C943A130E945B
:102680007B2C0E94BA190E943A160C9425138F9243
:102690009F92AF92BF92CF92DF92EF92FF920F93F1
:1026A0001F93CF93DF93CDB7DEB72A970FB6F89479
:1026B000DEBF0FBECDBF0E945C1681110E940613C3
:1026C00054E3852E52E0952E10E000E0A02E802FDE
:1026D0000E942C166C01F401E190F1904F01E81674
:1026E000F90609F45CC08091440281FD0E94351610
:1026F000C7018C259D25B12CEE24E394F12C9C017F
:102700002E213F21232B09F444C00E943713882334
:10271000A9F0BE82AF82CE20DF2081E0CD2809F46F
:1027200080E088870E94842C8160782F9A8789872F
:102730004E815F8168858A850E941707000F111FEF
:10274000F801EC5CFD4F80819181E826F926F18249
:10275000E0820E9452180E942C2B9091330289171C
:10276000A9F10E942C2B809333022A960FB6F8947D
:10277000DEBF0FBECDBFDF91CF911F910F91FF90B4
:10278000EF90DF90CF90BF90AF909F908F900C9480
:102790000507B394EE0CFF1CFBE0BF12B0CF0F5F38
:1027A0001F4F0430110509F091CF8FEF89838A8381
:1027B0001B820E94842C8160782F9D838C834981A9
:1027C0005A816B818D810E941707C3CF2A960FB65D
:1027D000F894DEBF0FBECDBFDF91CF911F910F9157
:1027E000FF90EF90DF90CF90BF90AF909F908F9031
:1027F000089590E080E008950895FC01EE0FFF1F1A
:10280000EE53FE4F859194910895CF93DF930E94EC
:102810001C15EC01811520E5920708F042C08115D6
:1028200030E4930708F0BDC0883E910528F5803E4E
:10283000910508F09DC0883A910588F4853A910584
:1028400008F08FC08130910509F492C0009709F417
:102850008FC0049708F08CC0D0E0C0E089C08F3BE7
:10286000910508F489C0805C9109C03CD105A0F3B2
:102870000E94FD13EC017CC08115904250F4C115FB
:1028800081E0D80708F074C0C03FD10528F3D065B7
:102890006FC0C11590E3D90708F079C0CE019F70D1
:1028A000E7CF811525E5920758F5811534E59307A3
:1028B00008F0A6C0811542E5940750F4C11581E5E2
:1028C000D80708F471C0DC2FCC27C16FD06A50C084
:1028D000982F969596959E0123703327C115D34561
:1028E00008F07FC0C1E0D0E002C0CC0FDD1F2A9508
:1028F000E2F720E2929FC0011124C82BD92B6FC0B0
:10290000C11589E5D807A8F4C11598E5D90708F0DD
:102910007CC0C11526E5D20708F09ECF8C2F0E94FF
:10292000B315C82FD0E0DC2FCC27CC27DF71D062C5
:102930001FC0C1153AE5D30708F46CC0CE0190560C
:102940008115904208F088CF8D2F8F710E94B315AA
:1029500090E0982F882788279F719C012C2BE901F4
:10296000E6CFC55AD0E0CC56DE4FC881D0E0D06467
:10297000CE01DF91CF910895C85AD0E0CC0FDD1F72
:10298000CA59DE4F0990D881C02DD464F1CFCE0151
:102990009927D3FF03C0EC01D86CEACFEC01D06CCF
:1029A000E7CFDF70D06AE4CFCE01E4E0969587955B
:1029B000EA95E1F783702C2F26952695237090E2F7
:1029C000299F90011124382B8C2F8370C1E0D0E017
:1029D00002C0CC0FDD1F8A95E2F7C22BD32BDC6837
:1029E000C7CFC1E0D0E002C0CC0FDD1F2A95E2F7CF
:1029F00030E2939FC0011124C82BD92BDA68B8CFDD
:102A0000D82FCC27C46FD06AB3CFDC2FCC27C06FB0
:102A1000D06AAECF8C2F8F700E94B31534E0D6955C
:102A2000C7953A95E1F7CF709C2FEC01D069A0CF04
:102A30000E940D200C94051482389105B1F1B0F478
:102A40008133910509F475C048F48932910509F480
:102A500069C08A32910509F473C0089585339105E0
:102A600009F459C08933910501F10895833E910518
:102A7000A9F138F4803E9105F9F0823E910549F1C3
:102A80000895863E9105A9F1873E9105C9F1843EDE
:102A9000910519F52091120321FF1FC080911103A8
:102AA00084FD14C087EE90E00895209111032370F7
:102AB000A1F080EE90E008952091110320FD47C021
:102AC0003091120330FF09C024FF44C090E080E041
:102AD00004C02091110322FDF7CF08952091110326
:102AE00022FD3BC03091120330FDE3CF24FFF5CF30
:102AF000EDCF2091110323FFF0CF24FDE7CFD2CFFC
:102B00002091110323FD2CC03091120331FFEECF31
:102B100084EE90E008952091110325FFDECF89E235
:102B200090E008952091110325FFD7CF85E390E031
:102B300008952091110326FFD0CF8AE290E00895F6
:102B40002091110326FFC9CF81E390E0089589E326
:102B500090E0089583EE90E0089582EE90E008956D
:102B600086EE90E008959091110392FF06C0282F01
:102B700028712830F9F4877F846093FF06C0282FDE
:102B800028712831F1F4877E84612091120320FF9F
:102B900006C0382F38713830D9F4877F816021FF23
:102BA00006C0282F28712831D1F4877E816194FDD9
:102BB000877E0895282F24712430F9F68B7F886052
:102BC000DCCF282F2471243101F78B7E8861DDCF83
:102BD000382F3171313019F78E7F8860E0CF282F80
:102BE0002171213121F78E7E8861E1CF80E0089547
:102BF0000C9455120E945C168FE39CE90197F1F743
:102C000000C000000E945C1680E00E942C1680FF2D
:102C100004C00E94F8150C94CF2C08950C94FA155A
:102C20000E945B12811102C00E94FF120E94661274
:102C3000809344020E946E129093120380931103BA
:102C40000E940E160E946A120E947B0B8091BD01A9
:102C50000C948E0B08950895E82FF0E0EE0FFF1FFF
:102C6000E55EFC4F808191810895089580EA8A9500
:102C7000F1F708950E946F03A3E1B3E011961C924F
:102C80001E92EBE1F3E01182108213961C921E92C9
:102C900012971382128215961C921E921497158217
:102CA000148217961C921E9216971782168284E041
:102CB0000E946F160C943205CF9383E193E00E943B
:102CC000AC03C82F282F44E06BE173E083E193E06D
:102CD0000E9470160E9438058C2FCF910895089598
:102CE000FF920F931F93CF93DF93F82E092F162F88
:102CF000D72FC42F222349F081E0809347020E94FE
:102D0000842C909346028093450280914702882349
:102D1000A1F080914502909146020E949C2C05975B
:102D200060F0EF2DF02FA12FBD2F90E080E0D0E0DC
:102D30008C179D0744F010924702DF91CF911F91AD
:102D40000F91FF900895219131912D933D9301961C
:102D5000EFCF0E94482C0E949A2E0E94B32E0E9410
:102D6000C52E0E943B13FBCF80914E0260916504FB
:102D70007091660480FF16C020910701269FC00154
:102D8000279F900D1124BC017695679576956795E0
:102D90006038710508F043C06115710509F441C040
:102DA000862F089581FF0BC020910701269FC00147
:102DB000279F900D1124BC0176956795E9CF82FF7E
:102DC00009C0809107019B01829FB001839F700D14
:102DD0001124DECF20914D022223D1F290910601E1
:102DE00080910701482F50E0291748F0CB01849FBC
:102DF000B001859F700D949F700D1124C9CF289F3D
:102E000090011124269FA001279F500D369F500D41
:102E10001124692F70E0CA010E943E34B9CF8FE7B8
:102E2000089581E0089580914E0280FF0CC060916A
:102E3000030170E075956795759567956115710546
:102E400049F1862F089581FF06C06091030170E06B
:102E500075956795F3CF6091030182FD0BC090914A
:102E60004C029923A1F06091020180910301961711
:102E700038F0682F70E06038710500F38FE708952F
:102E8000899FC001112470E00E945234F4CF61E0A8
:102E900070E0D7CF81E00895803F31F40E94B416EE
:102EA0008195809352020895813F19F40E94B416CF
:102EB000F8CF823F31F40E94B4168195809351027D
:102EC0000895833F19F40E94B416F8CF893F29F47E
:102ED0000E9413178093530208958A3F21F40E94A1
:102EE00013178195F7CF8B3F31F40E94131781950B
:102EF0008093540208958C3F19F40E941317F8CF61
:102F0000843F31F480915002816080935002089593
:102F1000853F21F4809150028260F7CF863F21F4F3
:102F2000809150028460F1CF873F21F4809150025C
:102F30008860EBCF883F21F4809150028061E5CF1B
:102F40008D3F31F480914E02816080934E0208954E
:102F50008E3F21F480914E028260F7CF8F3FB9F708
:102F600080914E028460F1CF90915102803F59F4DC
:102F70008091520287FF0DC01092520291110BC036
:102F800010924D0208C0813F81F4809152021816C0
:102F90009CF3992381F08091530290915402892BE4
:102FA00009F064C010924C020895823F49F497FFE3
:102FB000F0CF10925102809152028111ECCFE0CFFC
:102FC000833F19F41916ACF3E4CF20915302893FE3
:102FD00029F41216F4F610925302DBCF8A3F19F44B
:102FE00027FFD7CFF8CF209154028B3F29F427FF3A
:102FF000D0CF10925402CDCF8C3F19F41216CCF3DF
:10300000C8CF843F31F4809150028E7F809350026C
:10301000C0CF853F21F4809150028D7FF7CF863F4E
:1030200021F4809150028B7FF1CF873F21F4809172
:103030005002877FEBCF883F21F4809150028F7E32
:10304000E5CF8D3F31F480914E028E7F80934E020A
:10305000A0CF8E3F21F480914E028D7FF7CF8F3F1E
:1030600009F097CF80914E028B7FF0CF08950E9498
:10307000842C9C019091510280915202982B21F056
:1030800030934B0220934A02909153028091540254
:10309000982B21F030934902209348028FE492E06C
:1030A0000C94522BEF92FF920F931F93CF93DF93C9
:1030B00000D000D000D0CDB7DEB786E0EFE4F2E07C
:1030C000DE01119601900D928A95E1F7E090510290
:1030D000F09052020091530210915402109251024A
:1030E0001092520210925302109254028E2D8F2988
:1030F00091F080914A0290914B020E949C2CAC016D
:1031000090914D02992309F43FC0809108018417E2
:10311000150608F447C0802F812B91F0809148025A
:10312000909149020E949C2CAC0190914C029923F1
:1031300009F477C0809104018417150608F47FC054
:103140008091510290915202892B90915302892BC8
:1031500090915402892B11F00E94371886E0FE01ED
:103160003196AFE4B2E001900D928A95E1F7269690
:103170000FB6F894DEBF0FBECDBFDF91CF911F9188
:103180000F91FF90EF900895209109018AE0289F08
:10319000900111242417350708F0BDCF9F5F90934D
:1031A0004D0202C09F3FD1F7EE2059F00E94B416A5
:1031B0009FEF1E140CF491E0899F802D11248093C1
:1031C0005102FF2059F00E94B4169FEF1F140CF417
:1031D00091E0899F802D11248093520230915102F9
:1031E000332309F498CF20915202222309F493CF7C
:1031F00045EB3403C0011124992359F090935102F7
:1032000045EB240390011124332339F0309352020B
:1032100082CF81E080935102F3CF81E0809352020C
:103220007ACF209105018AE0289F9001112424176C
:10323000350708F085CF9F5F90934C0202C09F3FF7
:10324000D1F7002359F00E9413179FEF10160CF4CA
:1032500091E0899F802D112480935302112359F00E
:103260000E9413179FEF11160CF491E0899F802D97
:1032700011248093540230915302332309F460CF18
:1032800020915402222309F45BCF45EB3403C001A3
:103290001124992359F09093530245EB2403900194
:1032A0001124332339F0309354024ACF81E08093C4
:1032B0005302F3CF81E08093540242CF86E0EFE4E3
:1032C000F2E0DF011D928A95E9F710924D0210920B
:1032D0004C0210924E02089583E290E00E949C34CA
:1032E000863889F484E290E00E949C34803459F45A
:1032F00085E290E00E949C3491E0873B09F090E0E9
:10330000892F8170089580E0FCCFCF93C82F6FEF95
:10331000811166E883E290E00E94AA346FEFC11148
:1033200060E484E290E00E94AA346FEFC11167EB81
:1033300085E290E0CF910C94AA34089586E290E063
:103340000E949C34682F70E090E080E0089586E24F
:1033500090E00C94AA3480E00E94851960E070E04F
:10336000CB010E94A7190E942E1F0E94802081E09D
:103370000C9485190E949D190E946C19811102C03C
:103380000C94AB190895CF93FB01C281CC2309F1B2
:103390009C0122513F452031310520F582510E9488
:1033A0009020C0E08C2FCF91089581E00E94A10B66
:1033B00043E062E081E00E942905F3CF81E00E94B2
:1033C000AC0B43E062E081E00E942905EBCF82E094
:1033D000F6CF8031FFE59F0789F381319F45B9F32F
:1033E000C1E0E0CF8031EFE59E07F9F281319F45E2
:1033F000C9F682E0DBCF2FEFFC0120830895EF9226
:10340000FF920F931F93CF93DF93EC01062F8881D8
:103410002091690230916A02232B79F08E3F09F0E6
:1034200057C08981833020F08550833008F050C028
:10343000602FCE010E942E1D4BC08C3009F4A1C01C
:10344000D0F4843009F484C060F4823009F44AC0B6
:1034500008F071C08130C9F1602FCE010E94FB19C4
:1034600037C0863009F48AC008F47DC08A30A0F7DE
:103470008FEF88832DC0803109F4A0C0D8F48E303E
:1034800009F48BC008F481C080910A0190910B016E
:10349000892BF1F06B8170E06D317105C8F4898181
:1034A0009A81AE014C5F5F4F9827892798270E9429
:1034B00055200EC0823109F487C008F482C08331E0
:1034C00009F493C08E3F41F6B3CF198289E08A8315
:1034D000602FCE01DF91CF911F910F91FF90EF9060
:1034E0000C948E2D8981823071F0833079F0813097
:1034F00009F0B2CF0E94902C0E946C346A837B83C7
:103500008C839D83E5CF0E949E19F6CF80910A019E
:1035100090910B01892BE1F27E0110E0812F0E9436
:103520002C16F701928383831F5FF2E0EF0EF11CEC
:103530001430A1F7CDCF8981823009F08DCF6A8117
:103540007B818C819D810E946C340E94A719C0CF21
:103550004B816A8189810E94831E98278927982739
:103560009D838C83B5CF2C813D8132272327322741
:103570004B816A8189810E94A51EAACF0E942E1FBD
:10358000A7CF0E9429208983A3CF0E942B209827B0
:10359000892798279A8389839BCF6B8170E06D314F
:1035A000710508F095CF89819A81AE014C5F5F4F1C
:1035B0009827892798270E942E208ACF0E94802052
:1035C00087CF0E94711EDFCF6B8170E06D31710576
:1035D00008F07ECF89819A81AE014C5F5F4F9827BA
:1035E000892798270E94B31F73CF6B8170E06D31DC
:1035F000710508F06DCF89819A81AE014C5F5F4FF4
:103600009827892798270E94D91F62CF8F929F926F
:10361000AF92BF92CF92DF92EF92FF920F931F93E0
:10362000CF93DF93CDB7DEB72A970FB6F894DEBFFE
:103630000FBECDBF03E213E0F12CE12C84E8C82ECD
:103640008CE1D82E9EEAA92E9CE1B92E2BE8822E81
:103650002BE1922EF801D182C082B382A2829582A0
:103660008482F58AE48ABE016F5F7F4F8E2D0E94AF
:10367000DE1E892B29F489859A85F801938B828B2C
:10368000FFEFEF1AFF0A0A5E1F4F88E0E816F10409
:1036900009F72A960FB6F894DEBF0FBECDBFDF91B3
:1036A000CF911F910F91FF90EF90DF90CF90BF903F
:1036B000AF909F908F900895CF93DF9300D000D06C
:1036C0000F92CDB7DEB790935C0480935B048115B5
:1036D00020E2920748F40F900F900F900F900F90F8
:1036E000DF91CF910C9498048EEF89838A831B829B
:1036F0000E94842C8160782F9D838C8349815A811C
:103700006B818D810F900F900F900F900F90DF9134
:10371000CF910C9417070F931F93CF93DF938C01D6
:10372000EB0165E572E08C2F0E94DE1E892BA1F46F
:1037300080917B0490917C04019798F4DD27C15A15
:10374000DD4F8881F80110821882833041F180F4C6
:10375000813091F08230B9F0DF91CF911F910F91BC
:103760000895EFE9FFE03197F1F700C00000E4CFE2
:103770008430D1F0853081F78091550290915602C6
:10378000009751F306C0809157029091580200971C
:1037900099F3DF91CF911F910F910C945C1B809155
:1037A000590290915A02F3CF80915B0290915C0292
:1037B000009779F720915502309156028091570277
:1037C0009091580221153105D9F2009711F7C901DE
:1037D000E0CFCF93DF9300D000D00F92CDB7DEB70C
:1037E00090935C0480935B04811520E2920748F477
:1037F0000F900F900F900F900F90DF91CF910C943E
:1038000081048EEF89838A8381E08B830E94842CDC
:103810008160782F9D838C8349815A816B818D8152
:103820000F900F900F900F900F90DF91CF910C940D
:103830001707CF92DF92EF92FF921F93CF93DF9300
:10384000CDB7DEB72A970FB6F894DEBF0FBECDBF57
:10385000EBE0F4E080E5DF011D928A95E9F7E3ED06
:10386000F3E088E3DF011D928A95E9F78BE0C82E2B
:1038700084E0D82E7F0110E0F701D182C082BE0122
:103880006F5F7F4F812F0E94061F892B79F488E09C
:10389000FE013196D60101900D928A95E1F7898556
:1038A0009A85D70113969C938E931297BAE0CB0E0C
:1038B000D11CE7E0EE0EF11C1F5F1830E9F62A96E6
:1038C0000FB6F894DEBF0FBECDBFDF91CF911F9131
:1038D000FF90EF90DF90CF900895CF93DF93EC01AE
:1038E0000E94E91B80917B0490917C04019728F44D
:1038F000CE01DF91CF910C945C1BEFE9FFE0319793
:10390000F1F700C00000F2CF0F931F93CF93DF9326
:103910008C01862F65E572E00E94DE1E892BC9F4BA
:10392000C0915502D0915602209799F0F8018081FC
:10393000833069F4CE010E946D1CCE010E946D1C83
:10394000CE01DF91CF911F910F910C946D1C8430AB
:10395000B8F7DF91CF911F910F9108950F931F93A7
:10396000CF93DF938C01EB0165E572E08C2F0E9411
:10397000DE1E892B09F064C0FE01FF27D8018C915F
:10398000E15AFD4F8130D9F419969C9119979923EA
:1039900011F080830CC01A969C919923D1F382E098
:1039A000808380915702909158020097D9F48091BA
:1039B000550290915602009709F442C013C082301C
:1039C000E9F519968C91199781112DC01A968C9151
:1039D00081110EC083E080838091590290915A0238
:1039E000009719F1DF91CF911F910F910C94E91B72
:1039F00084E0808380915B0290915C02009791F754
:103A000080915502909156020097F9F00E946D1C2A
:103A10008091570290915802009721F780915502AA
:103A200090915602DFCF85E080838091550290917E
:103A30005602009729F00E946D1CF0CF86E080832B
:103A4000DF91CF911F910F9108958091570290912E
:103A50005802B1CF0E94061B0C94191CCF92DF9222
:103A6000FF920F931F93CF93DF93CDB7DEB72A97C3
:103A70000FB6F894DEBF0FBECDBF8C01603269F582
:103A8000DC011196EC911197EE3038F5F0E0EA5F29
:103A9000FA4C0C94663488E0EEE1F1E0DE01119618
:103AA00001900D928A95E1F780E2F80111928A95D2
:103AB000E9F784E0D8018C9311961C921197129625
:103AC0001C92129713961C92139788E0FE01319670
:103AD000149601900D928A95E1F72A960FB6F89404
:103AE000DEBF0FBECDBFDF91CF911F910F91FF9031
:103AF000DF90CF90089584E1F801808382E0818394
:103B000012821382EACF13968C911397682F70E07C
:103B1000762F662712968C91860F972F911D092E6E
:103B2000000CAA0BBB0B45E0880F991FAA1FBB1FF7
:103B30004A95D1F7AC01BD01405E5F4F6F4F7F4F9B
:103B4000481759076A077B0740F28431E2E09E0775
:103B5000A105B10510F64531F2E05F076105710579
:103B600020F044E152E060E070E0481B590BBC01DA
:103B70006E537E4FC8010E947334AFCF40E250E0D5
:103B80006FEF70E00E94853480910A01D8018C9318
:103B90008091690211968C93A0CF81E090E0909380
:103BA0006A028093690282E390E0909368028093B6
:103BB00067020E94842C91CF80910A01F8018083D2
:103BC00080916902818380916702828386CF40E27F
:103BD00050E0BC0112968D919C910E94D1217DCF25
:103BE000BC016F5F7F4F4FE150E0FC018281938108
:103BF0000E940322D8018C9370CFBC016C5F7F4F71
:103C00004CE150E0FC01828193810E942B22F2CF93
:103C10000E94922162CFFC0182818230F1F1E0F4B6
:103C2000882399F1813009F058CF13968C912AE0BE
:103C3000F22EFE0131966F01DF01EF2D1D92EA9504
:103C4000E9F7B6010E94DE1ED8018D93F6010190BE
:103C50000D92FA94E1F741CF833099F1843009F065
:103C60003CCF13968C919AE03496DE011196019028
:103C70000D929A95E1F7BE016F5F7F4F0E941A1F68
:103C8000F80180830E94191C28CF80E21D928A953A
:103C9000E9F788E08083818320CF13968C919AE0A6
:103CA0003496DE01119601900D929A95E1F7BE01CE
:103CB0006F5F7F4F0E94F21EF80180830E94061BF7
:103CC0000CCF13968C919AE0F92EFE0131966F017C
:103CD000DF01EF2D1D92EA95E9F7B6010E94061F5C
:103CE000B3CF84E0089550E0440F551F96E1699FDB
:103CF000400D511D112498E5899F400D511D11243F
:103D0000CA01879608950F931F93CF93DF93843052
:103D1000C8F46430B8F44B30A8F40E94731E8C01D0
:103D20000E949C34C82FD0E0DC2FCC27C80101961C
:103D30000E949C349E01282BC901DF91CF911F91D5
:103D40000F91089590E080E0F8CF0F931F93CF93E9
:103D5000DF93E9018430E0F46430D0F44B30C0F4F8
:103D600021153C4531F420910A0130910B01232BA0
:103D700079F00E94731E8C016D2F0E94AA346C2F63
:103D8000C8010196DF91CF911F910F910C94AA3435
:103D9000DF91CF911F910F9108958232910520F408
:103DA00089579E4F0C949C3480E00895823291058F
:103DB00020F489579E4F0C94AA3408959B018830B3
:103DC00070F49AE0899FB001112467557E4F4AE054
:103DD00050E0C9010E948C3490E080E008958FEF9C
:103DE0009FEF08959B01883070F49AE0899FB0019D
:103DF000112467557E4F4AE050E0C9010E94CE343D
:103E000090E080E008958FEF9FEF08959B01883048
:103E100070F49AE0899FB001112467507E4F4AE008
:103E200050E0C9010E948C3490E080E008958FEF4B
:103E30009FEF08959B01883070F49AE0899FB0014C
:103E4000112467507E4F4AE050E0C9010E94CE34F1
:103E500090E080E008958FEF9FEF08957F928F921A
:103E60009F92AF92BF92CF92DF92EF92FF920F9309
:103E70001F93CF93DF93CDB7DEB764970FB6F89457
:103E8000DEBF0FBECDBFA0900A01B0900B0181E054
:103E900090E090930B0180930A018AEBC82E80E09A
:103EA000D82E00E0760110E015C0F4012591349180
:103EB000472D612F802F0E94A51E82E0880E911C45
:103EC00073949BE07912F1CFE6E1EE0EF11C1F5FD7
:103ED000143019F04701712CE8CF0F5FF8E5CF0ED1
:103EE000D11C0430F9F60E9492211C861B861E8686
:103EF0001D86188A1F861A8A198A8FEA90E09C8B81
:103F00008B8B10E0BE01655F7F4F812F0E94F21EF8
:103F10001F5F1830B9F7CE0101967C018AE0F701E6
:103F200011928A95E9F710E0B701812F0E941A1FBC
:103F30001F5F1830C9F7B0920B01A0920A01649676
:103F40000FB6F894DEBF0FBECDBFDF91CF911F91AA
:103F50000F91FF90EF90DF90CF90BF90AF909F9028
:103F60008F907F900895EF92FF920F931F93CF93BE
:103F7000DF93EC018A017C01E60EF71ECE018796E5
:103F8000CE15DF0539F4DF91CF911F910F91FF908E
:103F9000EF900895C03621E0D20740F40E949C348F
:103FA000F80180830F5F1F4F2196E8CFF801108240
:103FB000F9CFCF92DF92EF92FF920F931F93CF939F
:103FC000DF938C016A018036914080F480E691E0B5
:103FD000801B910B8617970748F07801E60EF71EB5
:103FE000E801CE018796CE15DF0549F4DF91CF9128
:103FF0001F910F91FF90EF90DF90CF900895C03602
:1040000021E0D20740F4FE01E01BF10BEC0DFD1D99
:1040100060810E94AA342196E4CF462F2091690244
:1040200030916A02232B91F47E3F39F46E3F71F494
:1040300080915B0490915C040895843038F474306E
:1040400028F46B3018F4672F0C94831E90E080E006
:10405000089580E1089587EB91E00895EF92FF9233
:104060000F931F93CF93DF93EC018A017C01E60E3F
:10407000F71ECE01875B9D4FCE15DF0539F4DF912A
:10408000CF911F910F91FF90EF900895C73B21E0D2
:10409000D20740F40E949C34F80180830F5F1F4FC9
:1040A0002196E7CFF8011082F9CFCF92DF92EF92FD
:1040B000FF920F931F93CF93DF937C016A018C01D2
:1040C000060F171FEC01CE01875B9D4FC017D1076C
:1040D00049F4DF91CF911F910F91FF90EF90DF9006
:1040E000CF900895C73B21E0D20740F4FE01EE19BE
:1040F000FF09EC0DFD1D60810E94AA342196E3CFDB
:10410000CF93DF93C9E4D2E060E0CE010E94AA34ED
:104110002196C11584E0D807B9F7DF91CF910895B2
:10412000BF92CF92DF92EF92FF920F931F93CF93A4
:10413000DF9300D000D0CDB7DEB7F82E2FE02817E0
:1041400040F08FEF93E00E949C3409E412E0882352
:10415000D1F00F900F900F900F90DF91CF911F91A2
:104160000F91FF90EF90DF90CF90BF9008950115D1
:1041700044E0140771F3C8010E949C34811101C00E
:10418000FA940F5F1F4FF110F2CF19821A821B822F
:104190001C82BB24BA9478015FEFE51AF50AC801C6
:1041A0000E949C3489831A82882399F2813009F015
:1041B00047C0680182E0C80ED11CC7010E949C3430
:1041C000E82E8A83882329F2C6010E949C34F82EA7
:1041D0008FEF8E0D833068F46801E3E0CE0ED11CC2
:1041E000FB82FF2021F0CE0101960E948F068601FE
:1041F000D2CFF4E0EF12FBCF680124E0C20ED11C55
:10420000C80103960E949C34FF2009F4A2CF8823A2
:1042100009F49FCF8150990BB89E9001B99E300D43
:1042200011244F2D4150550BCA01820F931F019746
:10423000F0F2EFE9FFE03197F1F700C00000F7CFAF
:10424000CE0101960E948F066701D1CFEDE5F4E023
:10425000848195812AE030E0B9010E943E34609368
:1042600009018681809308018285809307018485F6
:104270008093060186859785B9010E943E3460933C
:1042800005018089809304018289809303018489D8
:1042900080930201089580915D0490915E040C94D6
:1042A000572A0F931F93CF93DF930DE514E0D0E0CF
:1042B000C0E0CE010E94CD1EF80161918F018617EA
:1042C00019F0CE010E94D61E2196C232D10589F77F
:1042D000DF91CF911F910F9108950F931F93CF936B
:1042E000DF930DE514E0D0E0C0E0CE010E94CD1ECA
:1042F000F80181938F012196C232D105B1F7CCED3F
:10430000D3E0FE0185919491009711F0FC0109958D
:104310002896F4E0C437DF07A1F7DF91CF911F9112
:104320000F910895EDE5F4E0128E138E2FEA30E040
:104330003183208385E0848F88E893E193838283AF
:104340006CE271E07583648342E350E057834683F7
:1043500085E090E0918780878AE090E0938782876C
:10436000A4E1B0E0B587A4877787668764E670E04C
:10437000718B608B68E070E0738B628B68E270E039
:10438000758B648B578B468B318F208F158E978F53
:10439000868F80E590E091A380A30E9451210C9428
:1043A0006D21EF92FF920F931F93CF93DF937C01C8
:1043B000EB018A016FEF70E0CE010E94853426ED9B
:1043C00033E0AEE6B4E090E080E0AC014E5F5F4FDA
:1043D0000417150788F0F90165917491E616F70640
:1043E00030F48C0F9D1FFC0171836083CA01285F2C
:1043F0003F4FA217B30749F7DF91CF911F910F915C
:10440000FF90EF900895DC01CB0126ED33E0F90138
:1044100065917491A617B70749F0285F3F4F64E094
:104420002E363607A1F78FEF9FEF0895B9016E5F23
:104430007F4FFB01A591B4914A175B07A0F3FB01E5
:1044400045915491F9013496659174910E947C34A0
:1044500090E080E00895CF93DF93C6EDD3E0FE01B6
:10446000259134918217930741F0289624E0CE36A7
:10447000D207A9F78FEF9FEF1DC0CE010296FC0176
:104480002591349142175307A8F3FC0145915491AB
:10449000FE013496859194910E947C340E945121B2
:1044A000FE01369685919491009711F0FC010995D3
:1044B00090E080E0DF91CF91089580917504909114
:1044C0007604089580917A048170089580917A0429
:1044D00086958170089580917A0482FB882780F9FF
:1044E000089580917A0483FB882780F9089580914C
:1044F0007304909174040895AF92BF92CF92DF92AB
:10450000EF92FF920F931F93CF93DF937C015B0198
:10451000C42FD22FFC0182818823F9F040936D02D1
:104520000E94842C90936C0280936B0280E28C0F2B
:10453000883008F061C0C77081E001C0880FCA955B
:10454000EAF7DF91CF911F910F91FF90EF90DF90ED
:10455000CF90BF90AF900C94240810916D0214136B
:1045600040C080916B0290916C020E949C2C6C0167
:10457000B701C5010E945D22C816D90690F5C0E2B8
:10458000CD0F1D17B9F080E2810F883040F417700D
:1045900081E001C0880F1A95EAF70E942B08C83005
:1045A00048F481E09D2F977001C0880F9A95EAF733
:1045B0000E942408802F0E941808C830E8F4D770A1
:1045C00081E001C0880FDA95EAF7DF91CF911F9162
:1045D0000F91FF90EF90DF90CF90BF90AF900C9431
:1045E0002B0880E28C0F883038F4C77081E001C05E
:1045F000880FCA95EAF7E9CFDF91CF911F910F910C
:10460000FF90EF90DF90CF90BF90AF9008950F9301
:104610009C01CB01233F4CE5340759F1A8F4283D18
:10462000FCE53F0701F1293D4CE53407D1F1273D79
:104630003C4591F406E221EE41EE67ED7CE50E94F7
:104640007C2280E00F910895253FFCE53F07E9F0CB
:10465000B0F0263F3C45F9F0FC018281882339F116
:1046600010926D02EFCF07E225EE45EE68ED7CE596
:10467000E6CF06E221EE40EE63EF7CE5E0CF07E215
:1046800025EE44EE64EF7CE5DACF06E221EE42EE61
:1046900065EF7CE5D4CF07E225EE46EE66EF7CE5DC
:1046A000CECF08E221E045EE69ED7CE5C8CF81E0A0
:1046B000C9CFCF93DF93EC01FB018281882309F4FA
:1046C00019C1C230FCE5DF07C0F1C6319CE5D9074E
:1046D00030F09E012A5F3C452930310570F50E947B
:1046E0006E129093120380931103C031ECE5DE0744
:1046F00009F4CFC008F05BC0C8308CE5D80709F4D6
:10470000B6C088F5C430ECE5DE0709F4A8C0C0F4F3
:10471000C2308CE5D80709F49CC0809111038260F7
:10472000C330DC4509F498C08091110390911203C5
:104730000E947C120E94560880E0DF91CF9108957C
:10474000809111038061C630ECE5DE0709F484C076
:10475000809111038860C730DC4508F47DC08091EA
:104760001103806279C0CC308CE5D80709F489C088
:1047700070F4809111038C60CA30ECE5DE0709F417
:104780006BC008F478C0809111038E7F65C0CE3075
:104790008CE5D80709F479C0809111038B7FCF3065
:1047A000DC4508F459C0809111038F7E55C0CB3F82
:1047B000ECE5DE0709F457C030F5C3318CE5D807C6
:1047C00009F46FC078F4C131ECE5DE0709F465C087
:1047D000C231DC4509F0A8CF0E9456088091110330
:1047E0008F773AC0C5318CE5D80709F462C008F468
:1047F00076C0809112038160CA3FDC4509F094CFF6
:104800008093120391CFCF3FFCE5DF0709F44DC041
:1048100088F4809112038D7FCD3F9CE5D90781F309
:10482000809112038E7FCE3FDC4550F380911203BE
:104830008360E6CFC130FDE5DF0709F459C008F415
:1048400044C080E0C230DD4509F06ECF0E94011304
:104850006BCF8091110381608093110365CF8091AC
:1048600011038460F9CF809112038260C9CF8091D7
:1048700011038064F1CF0E94560880911103806873
:10488000EBCF809111038D7FE7CF80911103877F5C
:10489000E3CF809111038F7DDFCF809111038F7B58
:1048A000DBCF80911103837FD7CF809112038C7F60
:1048B000A7CF8091110382FB992790F921E09227DD
:1048C00090FB82F990FB83F9C7CF80911203982F58
:1048D000909591708E7F892B90FB81F991CF0E94EA
:1048E000560890911103892F97FB87F98058B4CF10
:1048F00081E0ACCF81E021CFCF93DF93EB01863114
:104900009C4509F03BC00E945911982F9A7A20913A
:10491000770420FF04C0382F347409F090E021FFA1
:1049200004C0382F317109F090E022FF04C0382F05
:10493000387809F090E023FF03C0827209F090E01C
:104940008A81882389F081E0911101C080E0809301
:104950006E0289E2911185E30E94DC100E94D11160
:1049600080E0DF91CF91089580916E02811104C0A3
:1049700089E20E94E310F2CF85E3FBCF81E0F1CF23
:1049800008950F931F93CF93DF938091DA02E09104
:104990006F021CE081111AC0DF91CF911F910F911E
:1049A000089501E00E0F00936F02CE2FD0E0E19F3B
:1049B000F0011124E658FD4F83819481892B29F061
:1049C0008081918189238F3FE9F4E02F8091DA0281
:1049D000E81738F31092DA0210926F02DDCF1896C2
:1049E0008D919C918F3F9807D1F061E00E94C02487
:1049F0001C9FF0011D9FF00D1124E658FD4F1482FD
:104A00001382E3CF1C9FD0011D9FB00D1124A65827
:104A1000BD4F16968D919C911797892B01F320819C
:104A200031814281538164817581868197810E94A1
:104A30003C10DECF1092DC021092DB0220910D01BF
:104A400030910E01E3EDF3E090E080E028173907A4
:104A500009F408954581411102C01482168201961D
:104A60003796F4CFDC016091780280917902962F1D
:104A7000891301C00895292F30E0F901EE0FFF1FBF
:104A8000E059FD4F408151814A175B07A1F487E04F
:104A90008A9FA0018B9F500D11244D525C4F81E0E5
:104AA000FA0184839613E6CF2F5F3F4F237033279D
:104AB0002093780208952F5F3F4F922F9370D8CFA5
:104AC0006F927F929F92AF92BF92CF92DF92EF92BE
:104AD000FF920F931F93CF93DF93DB0114962C91DA
:104AE0001497211169C0A090DA02EAE7F2E030E001
:104AF00020E0B12C66246394712C2A1508F047C07D
:104B0000C284D384ED90FC9011976FEF7FEF912CCE
:104B1000492D50E08A01000F111F0E0D1F1DE801E5
:104B2000088119810115110531F0C016D10609F46B
:104B3000BA019394EDCF6F3F7607D1F1E30102C044
:104B4000CC0FDD1F6A95E2F7BC2AB30102C0660FE5
:104B5000771F9A94E2F7AB0141505109B41615063C
:104B600029F512964D915C9113976CE0629FF001CC
:104B7000639FF00D1124E658FD4F578346832EEFB7
:104B8000208321839187808721E015962C93DF91E4
:104B9000CF911F910F91FF90EF90DF90CF90BF903A
:104BA000AF909F907F906F900C9432251482138267
:104BB0002F5F3F4F3C96A1CFDF91CF911F910F9177
:104BC000FF90EF90DF90CF90BF90AF909F907F903D
:104BD0006F9008951F93CF93DF93C091780217E0F1
:104BE000809179028C1307C00E94C124DF91CF917C
:104BF0001F910C941A25D0E0FE01EE0FFF1FE05923
:104C0000FD4F80819181189FB001199F700D112473
:104C10006D527C4F0E9460252196C370E1CF0F93A7
:104C20001F93CF93DF93DC012D913C91119740E0CE
:104C300090E080E0E82FF0E0EE0FFF1FE20FF31F9F
:104C4000C081D1812097B9F0FB010081118190E0F2
:104C500005C0CE17DF0709F441E09F5FE92FF0E0C0
:104C6000EE0FFF1FE00FF11F0190F081E02D309754
:104C700081F78F5FDFCF442349F0981708F4DB01F9
:104C8000CD01DF91CF911F910F910895B0E0A0E089
:104C9000F7CF80910C01882341F18091DD02909142
:104CA000DE02009711F10E949C2C2091DB023091D2
:104CB000DC0228173907C8F49091780280917902B4
:104CC000981759F00E94EA251092DC021092DB023C
:104CD0001092DE021092DD0208950E94C12410920B
:104CE000DE021092DD020C941A2508951092DE0265
:104CF0001092DD0210920C0180917902809378026B
:104D00000E941A250C94C12480910C0181110C94ED
:104D1000762681E080930C0108952F923F924F9266
:104D20005F926F927F928F929F92AF92BF92CF923B
:104D3000DF92EF92FF920F931F93CF93DF93CDB744
:104D4000DEB72A970FB6F894DEBF0FBECDBF6C0159
:104D50002B01FB011281873FFCE59F07F9F411232A
:104D600021F181E080930C01812F2A960FB6F894EF
:104D7000DEBF0FBECDBFDF91CF911F910F91FF908E
:104D8000EF90DF90CF90BF90AF909F908F907F90EB
:104D90006F905F904F903F902F900895883F2CE543
:104DA000920709F04DC0111148C003ED13E0F12C3A
:104DB000E12C1986AA24A394B12C80910D01909125
:104DC0000E01E816F90608F445C0F2018281882335
:104DD00009F466C1F985FF2309F462C10E94842C9D
:104DE0009093DE028093DD028091DA02883008F52C
:104DF00091E0980F9093DA0298E0F201DE011196AB
:104E000001900D929A95E1F72CE0829FC001112448
:104E100086589D4F28E0FE013196DC0101900D92ED
:104E20002A95E1F72FEF3FEFFC0131872087D386EA
:104E3000C28611E0F9851F2797CF0E94762694CF6E
:104E4000893F9C4509F0B1CF112309F4AECF0E94F0
:104E500084268ACFF8012081318166246A94762CD9
:104E6000212C822D90E0FC01EE0FFF1FE20FF31FBB
:104E7000408151814115510531F0C416D50609F420
:104E80003C012394EECF312CFFEF6F167F0609F41F
:104E900048C0F801448130900C01832D411180E01D
:104EA000F82FF1703F2EF2018281882309F496C019
:104EB000332009F493C0B801C7010E9477224C0146
:104EC000F8018581811113C0950101C0220F6A94F8
:104ED000EAF78681822B86838091DB029091DC0247
:104EE0008815990520F49092DC028092DB02C501BE
:104EF00002C0880F991F2A94E2F70197F8012681D2
:104F00002817190671F48091DD029091DE02009756
:104F100089F00E949C2C8816990660F421E0F80123
:104F20002483F985F329F9872FEFE21AF20A095F42
:104F30001F4F43CF20907802309179023A8790E05A
:104F400080E0EA852E1215C08017910751F3822C5C
:104F5000912CF401EE0FFF1FE059FD4FF182E0822A
:104F6000FFEF8F1A9F0A23E0822299248092790210
:104F7000D8CF822C912CF401EE0FFF1FE059FD4F8A
:104F80002081318147E0429FC001439F900D112451
:104F9000FC01ED52FC4F3F01B801CF010E940F26EA
:104FA0000097A9F021E0FC0124838017910709F400
:104FB000B8CF2091780222120AC06816790639F417
:104FC00094012F5F3F4F23703327209378023FEFE8
:104FD000831A930A482D4370242EB3CFF80195808D
:104FE000868190E091101EC0950102C0220F331FF0
:104FF0002A94E2F7215031092817390731F4442364
:1050000009F44CC0C7010E943225C50101C0880FB8
:105010006A94EAF7982F9095F80186818923868310
:10502000392C7FCF9C01062C02C0359527950A9418
:10503000E2F7A90141705527BC016150710986232F
:105040009723892B39F5452B29F182819381892B6F
:10505000E1F01B821C821D821E82FEEFF983FA831F
:105060000E94842C8160582F9D838C83F80182815B
:1050700093818F83988729813A814B816D817E81CD
:105080000E943C10F8011582C0CF60E0C7010E9469
:10509000C024F8CFF22FF1709F2EB7CF932CB5CF4D
:1050A0009091780280917902981719F00E94EA2570
:1050B000C0CE0E94C1241092DE021092DD020E9436
:1050C0001A25B7CECF93DF93EC0181E0898B8F81D6
:1050D0000E945C1188850E946F110E94D111EA81A3
:1050E000FB81309739F06C897D89CE010696DF917E
:1050F000CF910994DF91CF910895EF92FF920F9392
:105100001F93CF93DF93EC018A85811134C0EB802C
:10511000FC8087E5F81A26E12E9DC0012F9D900D99
:105120001124DC01AD5DBC4F1496ED91FC911597F7
:10513000309731F054966D917C91875D9C4F099525
:1051400086E18E9D80018F9D100D11240D5D1C4FF9
:10515000F80187810E946211F80180850E94751113
:105160000E94D111188219861B861E821D82109200
:10517000E0021092DF02DF91CF911F910F91FF901B
:10518000EF900895DF92EF92FF920F931F93CF93CA
:10519000DF937C01FB018281882391F080910F01D4
:1051A0008F3F71F0C3E2D3E010E000E0DD24D39440
:1051B00080910F01082E000C990B8017910744F481
:1051C000DF91CF911F910F91FF90EF90DF900895A5
:1051D0008E818823D9F089859A858E159F0539F4AB
:1051E0008091DF029091E0028E159F0579F0DF86B5
:1051F000FC86EB868989811103C0CE010E9462285A
:10520000CE0106960E947D280E947C110F5F1F4FE1
:105210006696CECFEF92FF920F931F93CF93DF93BB
:105220007C0197558F3F910509F0D8F520910F012A
:10523000022E000C330B2817390714F480930F014A
:10524000FB01228136E1389F8001399F100D112426
:10525000E801CD5DDC4F288B92818E81992349F145
:10526000FA86E9868F5F8E830E94842C9E878D87C5
:105270000E948F118F830E94591188870E946C11A0
:105280009885892B8887E881F981309731F06C897E
:105290007D89C801875D9C4F0995F092E002E092FC
:1052A000DF0281E0DF91CF911F910F91FF90EF908E
:1052B00008958823B1F38989882399F3C801875D0C
:1052C0009C4F0E947D28EDCFCF92DF92EF92FF920C
:1052D0000F931F93CF93DF9380910F0110E006E1AE
:1052E0008F3FF1F5DF91CF911F910F91FF90EF90DC
:1052F000DF90CF9008950E9DF0010F9DF00D1124C9
:10530000ED5DFC4FC288D388C114D10439F470E03C
:1053100060E0818592850E945D226C010E9DE00116
:105320000F9DD00D1124CD5DDC4F8E818823B9F007
:105330008D859E850E949C2CC816D90680F4109FEE
:10534000700111248989811105C0C7018D5D9C4FB1
:105350000E946228C701875D9C4F0E947D281F5FC5
:10536000E12EF12C80910F01082E000C990B8E1567
:105370009F050CF6B7CFFF920F931F93CF93DF9348
:105380008C01EB01F42E8091100182FF4AC08B7FCB
:10539000809310018091E3029091E4029B01281B0D
:1053A000390BC90120911101309112018217930725
:1053B000B8F48091E1020E948407809110018D7FF2
:1053C0008093100180917B0490917C04019710F5EB
:1053D0008091E1020E94D20782E00E9475112BC0E9
:1053E00082E00E946F118091E1020E948407809107
:1053F00010018260809310018091780485FFE2CFD4
:1054000086FDE0CFFF20F1F2DF91CF911F910F9148
:10541000FF900895EFE9FFE03197F1F700C0000039
:10542000D5CF802F0E94D2078091E1029091E202B5
:105430008017910789F20E94D111D093E402C093A2
:10544000E302E2CF8091780480FF1DC080911001BB
:1054500082FF19C00E94842C2091E3023091E40263
:10546000AC01421B530B9A01409111015091120162
:105470002417350740F041E0BC018091E102909192
:10548000E2020C94BB29089590911001892F8E7F20
:1054900090FF81608093100182E00C9475118091DF
:1054A00010018E7F8093100182E00C94751190930F
:1054B00012018093110108958832910538F48E31DC
:1054C0009105E8F40497A0F480E0089589339105EC
:1054D00058F48D32910510F48B97B1F780917804D0
:1054E00082FB882780F908C084369105B9F3ECCF98
:1054F000809178048295817091E089270895809148
:10550000780483FB882780F9F7CFCF92DF92EF9260
:10551000FF920F931F93CF938C016B0180917804BE
:1055200080FD0AC0C1E08C2FCF911F910F91FF9099
:10553000EF90DF90CF9008950E94842C7C01F601BB
:10554000C281CC2329F18091100182FF06C040E086
:10555000B70190E080E00E94BB2982E00E947511B3
:105560000B31FCE51F0759F00C314CE5140769F0CD
:105570000A315CE5150761F40E94442AD4CF80917A
:105580001001816080931001CECF0E944F2ACBCFB3
:10559000B601C8010E945C2A882321F2F601C2816B
:1055A000CC2309F44EC08091100180FFBBCF8091C5
:1055B000780481FF15C08091780485FD16C0109392
:1055C000E2020093E102F092E402E092E3028091B1
:1055D000100184608093100182E00E9439122FC074
:1055E0000E945911882339F39DCF2091E302309115
:1055F000E402A701421B530B9A0186FD04C080916F
:10560000100181FDDCCF2F3A3105C8F68091E1020F
:105610009091E2020817190791F68091100181FB21
:10562000CC27C0F981FD04C0802F0E9484077BCF66
:1056300082E00E946F118091E1020E948407C0E025
:1056400072CF40E0B701C8010E94BB296CCF909394
:10565000EA028093E9020895E091E902F091EA02FA
:10566000309721F00190F081E02D099480E00895B9
:10567000E091E902F091EA02309799F020911D0142
:10568000222359F02091110327FF07C0DC012C9140
:1056900011962C93119725E02C930280F381E02D35
:1056A00009940895E091E902F091EA02309739F007
:1056B00022E0DC012C930480F581E02D099408950B
:1056C0002091E7023091E8022817390771F0909392
:1056D000E8028093E702E091E902F091EA02309754
:1056E00021F00680F781E02D099408952091E502CC
:1056F0003091E6022817390771F09093E602809303
:10570000E502E091E902F091EA02309721F000848D
:10571000F185E02D09940895FC01329680911D01D8
:10572000882321F0809111039EE187FF96E080E0BD
:10573000915008F4089521912223D1F38F5FF8CF7F
:10574000662301F120911D012223F1F02091110324
:1057500027FF1AC0462F4695469546954E3190F440
:10576000677021E030E002C0220F331F6A95E2F734
:10577000840F911DFC01828190E02823392381E070
:10578000232B69F480E00895FC013296089621915C
:10579000261721F0E817F907D1F7F4CF81E0089533
:1057A0009C01FC0132969FEF80E04191461751F039
:1057B0009F3F19F4411101C0982F8F5F8630A9F7E0
:1057C0009F3F09F40895290F311D97FD3A95F9017E
:1057D00062830895FC01329608962191261303C036
:1057E000DF0111971C92E817F907B9F70895E62F22
:1057F000E695E695E695EE3168F4E80FF92FF11D90
:10580000677021E030E001C0220F6A95EAF78281DB
:10581000822B82830895E62FE695E695E695EE3194
:1058200070F4E80FF92FF11D677021E030E001C03E
:10583000220F6A95EAF72095828128232283089512
:1058400020911D01222329F02091110327FD0C94A2
:10585000F72B0C94D02B20911D01222329F02091AD
:10586000110327FD0C940B2C0C94EA2BFC013296AF
:1058700080911D01882351F08091110387FF06C09C
:105880008EE1DF011D928A95E9F7089586E0F9CF50
:10589000089508950C94492C0E9456080E942C2BC0
:1058A0000E9405070C944A2C1F921FB61F921124C8
:1058B0008F939F93AF93BF938091EB02811113C09D
:1058C00080917F0490918004A0918104B091820422
:1058D0004196A11DB11D80937F0490938004A093F5
:1058E0008104B0938204BF91AF919F918F911F90DB
:1058F0001FBE1F90189582E084BD93E095BD9AEF7E
:1059000097BD80936E0008952FB7F89480917F041F
:1059100090918004A0918104B09182042FBF0895DA
:105920002FB7F89460917F04709180048091810476
:10593000909182042FBF08959C014FB7F8948091F5
:105940007F0490918004A0918104B09182044FBFA4
:10595000821B930B089578941F921FB61F921124F7
:105960008F939F93AF93BF9380917F049091800416
:10597000A0918104B09182040196A11DB11D809374
:105980007F0490938004A0938104B0938204BF911C
:10599000AF919F918F911F901FBE1F90189581E02E
:1059A0008093E00080E28093D8001092C9008FE1DC
:1059B0009EE40197F1F700C0000087E090EBDC0166
:1059C0008093900490939104A0939204B0939304D5
:1059D00088E19CE00FB6F894A895809360000FBE14
:1059E00090936000FFCF9093A7018093A601089544
:1059F00080910F03089590918704943029F5809346
:105A0000EC027093EE026093ED029093E9008FEF49
:105A10009091E800815095FD06C095ED9A95F1F7BB
:105A200000008111F5CF8091E80085FF0DC050E0A6
:105A300040E063E070E08CEE92E00E945E2F809187
:105A4000E8008E778093E8000895BC0184E00C9410
:105A5000FB2CBC0183E00C94FB2C9C0184E0809324
:105A6000E9009FEF8091E800915085FD06C085ED2B
:105A70008A95F1F700009111F5CF8091E80085FF3C
:105A80000CC050E040E066E070E0C9010E945E2F6B
:105A90008091E8008E778093E8000895CF93DF939C
:105AA000EC0180911D018823B1F18091110387FFE2
:105AB00032C060E284E08093E9008FEF9091E800CB
:105AC000815095FD06C095ED9A95F1F70000811182
:105AD000F5CF8091E80085FF1BC080911D0170E02B
:105AE00050E040E0811104C050E040E068E070E028
:105AF000CE010E945E2F8091E8008E778093E800AF
:105B000080E2FE01AFEEB2E001900D928A95E1F7DE
:105B1000DF91CF91089568E081E0CDCFCF93FC0174
:105B2000603221F580918704843001F5C091E9004D
:105B3000CF702091EC00922F917020FD90E8C92B3E
:105B400082E08093E9008091E80080FF0CC050E083
:105B500040E060E270E0CF010E945E2F8091E8009B
:105B60008E778093E800CF70C093E900CF910895BD
:105B700080918604811109C00E943D310E949A31B2
:105B80008091E20084608093E20008951092860480
:105B90000895089508950C944C2C42E061EC81E046
:105BA0000E94B93042E261EC84E00E94B93042E2E6
:105BB00061EC82E00E94B93042E260EC83E00C9438
:105BC000B93080918904833009F461C030F48130A8
:105BD000D1F1823009F49DC008958A3009F489C05A
:105BE0008B3009F46FC0893009F050C0809188046F
:105BF000813209F04BC080918C0490918D04009704
:105C000019F0029709F042C08091E800877F8093E5
:105C1000E8008091E80082FF35C09091F300809108
:105C2000F200029729F48091F1008B7F813021F4FA
:105C30008091F10080930F038091E8008B7780932F
:105C4000E8000C94ED3080918804813AF9F4809159
:105C5000E800877F8093E80080918C0490918D0408
:105C6000892B61F460E28FEE92E070E00E94FC2FDD
:105C70008091E8008B778093E800089560E090E0E1
:105C800080E0F3CF809187048111C3CF0895809184
:105C90008804813AD9F780918C0490918D04892BE6
:105CA000A9F78091E800877F8093E8008091E80061
:105CB00080FFFCCF80911D018093F1008091E8006E
:105CC0008E77BDCF80918804813201F780918C045A
:105CD00090918D04892BD1F68091E800877F809385
:105CE000E8000E94ED3080918A0480931D010C949D
:105CF000560880918804813249F68091E800877FB8
:105D00008093E8000E94ED3080918B048093100313
:105D1000089580918804813A09F0B8CF8091E80015
:105D2000877F8093E8008091E80080FFFCCF80911E
:105D30001003C2CF84B7877F84BF0FB6F894A895AD
:105D400080916000886180936000109260000FBEB7
:105D500080E890E00FB6F894809361009093610022
:105D60000FBE0C9427130E943D310E949A31E2EE3F
:105D7000F0E080818460808378940E9423340E94C4
:105D80003F1383E191E00C94272BCF93DF93CDB7A2
:105D9000DEB7A0970FB6F894DEBF0FBECDBF0E944E
:105DA000471380918704843009F583E08093E900EC
:105DB0008091E80082FF1AC08091E80090E085FFA2
:105DC00009C050E040E060E270E0CE0101960E9420
:105DD000AD2F91E08091E8008B778093E8009923C4
:105DE00029F060E2CE0101960E94FF19A0960FB63D
:105DF000F894DEBF0FBECDBFDF91CF9108950C9414
:105E0000012F292F33272330310521F168F4213068
:105E1000310509F449C02230310509F44AC090E047
:105E200080E030E020E029C02132310581F12232CA
:105E30003105A9F76330710590F7FB01EE0FFF1FE5
:105E4000E656FE4F2081318169567E4FFB018081ED
:105E500090E013C099278130910599F0009741F0A7
:105E60008230910589F00397D1F6EEE6F4E002C0A6
:105E7000ECEBF4E0849190E09F01FA013183208300
:105E80000895E8E9F4E0F6CFECE8F4E0F3CF63300E
:105E9000710528F6660F771FFB01E056FE4F208143
:105EA000318189E090E0E9CF82E190E02BE135E0BB
:105EB000E4CF8BE590E020EC34E0DFCFAF92BF92EF
:105EC000CF92DF92FF920F931F93CF93DF936C01DA
:105ED000EB018A010E940C31F82E811123C00115BB
:105EE000110539F0F80180819181C81BD90BC80ECA
:105EF000D91EB12CA12C2097A9F08091E80085FD36
:105F000022C08091E8008E778093E800011511058A
:105F1000A1F0F80180819181A80EB91EB182A08202
:105F200085E0F82E8F2DDF91CF911F910F91FF907B
:105F3000DF90CF90BF90AF9008950E940C318823DE
:105F4000D1F2F82EEFCFF60181916F018093F1002D
:105F50002197FFEFAF1ABF0ACECFAF92BF92CF9279
:105F6000DF92FF920F931F93CF93DF936C01EB01AE
:105F70008A010E940C31F82E811123C001151105F0
:105F800039F0F80180819181C81BD90BC80ED91E48
:105F9000B12CA12C2097A9F08091E80085FD22C0AA
:105FA0008091E8008B778093E80001151105A1F03E
:105FB000F80180819181A80EB91EB182A08285E08E
:105FC000F82E8F2DDF91CF911F910F91FF90DF90D1
:105FD000CF90BF90AF9008950E940C318823D1F2EA
:105FE000F82EEFCF8091F100F60181936F01219798
:105FF000FFEFAF1ABF0ACECFFC0180918E049091C3
:106000008F0486179707A0F06115710529F4909108
:10601000E8009E779093E80090E06115710551F4D7
:10602000911108C08091E80082FF34C080E008959B
:10603000BC01F2CF809187048823C1F18530C1F182
:106040008091E80083FD30C08091E80082FDEACFB6
:106050008091E80080FFE1CF8091F3002091F20071
:10606000382F6115710519F02830310558F091E08D
:106070002830310509F090E02091E8002E77209338
:10608000E800CBCF81918093F100615071092F5FBF
:106090003F4FE7CF80918704882341F0853041F05E
:1060A0008091E80083FFBECF81E0089582E00895EB
:1060B00083E00895FC0180918E0490918F048617EF
:1060C0009707A0F06115710529F48091E8008E779B
:1060D0008093E80090E06115710551F4911108C0BA
:1060E0008091E80082FF35C080E00895BC01F2CFC6
:1060F000809187048823C9F18530C9F18091E80037
:1061000083FD31C08091E80082FDEACF8091E800F4
:1061100080FFE1CF8091F3002091F200382F6115CC
:10612000710519F02830310558F091E0283031051B
:1061300009F090E08091E8008E778093E800CBCF63
:1061400084918093F1003196615071092F5F3F4F28
:10615000E6CF80918704882341F0853041F080911B
:10616000E80083FFBDCF81E0089582E0089583E0D9
:106170000895982F973028F08F708093E90081E080
:1061800008959093E900242F762F50E0981731F06E
:106190007091EC002091ED005091F00021FD02C0C3
:1061A0009F5FE8CF3091EB003E7F3093EB00309162
:1061B000ED003D7F3093ED003091EB003160309386
:1061C000EB007093EC002093ED005093F0002091D1
:1061D000EE0027FDE5CF80E008958091880487FFD9
:1061E00013C08091E80082FF06C08091E8008B77A1
:1061F0008093E80004C0809187048111F2CF089554
:10620000809187048823D9F38091E80080FFF8CF3C
:106210008091E8008E77ECCF2091E4003091E5008A
:1062200095E6A9012091EC00822F817020FF06C025
:106230008091E80080FF06C080E008952091E8008A
:1062400022FD1AC080918704882389F0853089F067
:106250008091EB0085FD0FC02091E4003091E500B6
:1062600042175307F9F29150E1F684E0089582E075
:10627000089583E0089581E008950E94AB310E9463
:10628000B331E0EEF0E0808181608083E8EDF0E002
:1062900080818F77808319BCA7EDB0E08C918E7FD1
:1062A0008C9380818F7E80831092860408950F9353
:1062B0001F93CF93DF930E94AB310E94B331C8ED9F
:1062C000D0E088818F7788838881806888838881FF
:1062D0008F7D888319BC10928704109283041092DA
:1062E00085041092840400EE10E0F80180818B7F19
:1062F000808388818160888342E060E080E00E9442
:10630000B930E1EEF0E080818E7F8083E2EEF0E054
:10631000808181608083808188608083F8018081B2
:106320008E7F8083888180618883DF91CF911F91E8
:106330000F910895E8EDF0E080818F7E8083E7ED96
:10634000F0E080818160808384E082BF81E080937F
:1063500086040C945731E8EDF0E080818E7F8083D5
:106360001092E20008951092DA001092E100089570
:106370001F920F920FB60F9211242F933F934F93BA
:106380005F936F937F938F939F93AF93BF93EF939D
:10639000FF938091E10082FF0BC08091E20082FFB9
:1063A00007C08091E1008B7F8093E1000E9422343E
:1063B0008091DA0080FF19C08091D80080FF15C05D
:1063C0008091DA008E7F8093DA008091D90080FF7F
:1063D00096C080E189BD82E189BD09B400FEFDCF90
:1063E00081E0809387040E94B82D8091E10080FFB6
:1063F00019C08091E20080FF15C08091E2008E7F7D
:106400008093E2008091E20080618093E2008091BD
:10641000D80080628093D80019BC85E080938704FF
:106420000E94CA2D8091E10084FF2BC08091E20080
:1064300084FF27C080E189BD82E189BD89B5982F9D
:10644000917080FFFBCF8091D8008F7D8093D80022
:106450008091E1008F7E8093E1008091E2008F7E49
:106460008093E2008091E20081608093E20080915D
:106470008304882309F449C084E0809387040E9440
:10648000CB2D8091E10083FF29C08091E20083FF42
:1064900025C08091E100877F8093E10082E08093B6
:1064A0008704109283048091E1008E7F8093E10045
:1064B0008091E2008E7F8093E2008091E200806113
:1064C0008093E20042E060E080E00E94B930809179
:1064D000F00088608093F0000E94C92DFF91EF9139
:1064E000BF91AF919F918F917F916F915F914F91EC
:1064F0003F912F910F900FBE0F901F90189519BCD0
:10650000109287040E94C62D70CF8091E30087FD12
:1065100093E090938704B3CF1F920F920FB60F9220
:1065200011242F933F934F935F936F937F938F9398
:106530009F93AF93BF93CF93DF93EF93FF93D0914C
:10654000E900DF708091EC00C82FC17080FDC0E8C9
:106550001092E9008091F000877F8093F00078949A
:106560000E94D0321092E9008091F0008860809300
:10657000F000CD2BCF70C093E900FF91EF91DF9138
:10658000CF91BF91AF919F918F917F916F915F91CB
:106590004F913F912F910F900FBE0F901F90189524
:1065A0001F93CF93DF93CDB7DEB7AA970FB6F894BA
:1065B000DEBF0FBECDBF88E894E02091F100FC0162
:1065C0002193CF01F4E080399F07B9F70E94E12DB4
:1065D0008091E80083FF1EC1809188049091890416
:1065E0009A3008F017C1E92FF0E0EC5EFA4C0C94F9
:1065F0006634803899F0823809F00CC180918C049F
:106600008F70873008F006C18093E9008091EB001D
:1066100085FB882780F91092E90006C080918404E8
:1066200090918504911182609091E800977F9093FA
:10663000E8008093F1001092F1008091E8008E77DD
:10664000E5C0882309F4D3C0823009F0E3C080910B
:106650008A048111D6C080918C048F702FEF280F8F
:10666000263008F0D7C08093E9002091EB0020FF8E
:10667000C8C0933031F48091EB0080628093EB00CE
:10668000C0C09091EB0090619093EB0021E030E06E
:1066900001C0220F8A95EAF72093EA001092EA00DF
:1066A0008091EB008860EACF8111B4C010918A0418
:1066B0001F778091E3008078812B8093E3008091A5
:1066C000E800877F8093E8000E94ED308091E80029
:1066D00080FFFCCF8091E30080688093E30082E03C
:1066E000111183E08093870495C08058823008F0B0
:1066F00091C080918A0490918B048C3D23E0920795
:10670000A1F583E08A838AE289834FB7F894DE019A
:10671000139620E03EE051E2E32FF0E05093570063
:10672000E49120FF03C0E295EF703F5FEF708E2F82
:1067300090E0EA30C0F0C7968D939D932F5F24318F
:1067400059F74FBF8091E800877F8093E8006AE2A5
:1067500070E0CE0101960E94FC2F8091E8008B77BB
:106760008093E80057C0C096E7CF60918C04709189
:106770008D04AE014F5F5F4F0E94FF2EBC01892B3D
:1067800009F448C09091E800977F9093E8008981D0
:106790009A810E945A30E1CF8038E1F58091E8007B
:1067A000877F8093E800809183048093F10045CF38
:1067B000811130C090918A04923060F58091E80098
:1067C000877F8093E800909383040E94ED3080914E
:1067D0008304882311F084E005C08091E30087FDE5
:1067E000FACF81E0809387040E94CD2D13C0809161
:1067F0008A04813079F481E0933009F080E080935D
:1068000085041092E9008091E800877F8093E8007A
:106810000E94ED308091E80083FF0AC08091E8007B
:10682000877F8093E8008091EB0080628093EB008B
:10683000AA960FB6F894DEBF0FBECDBFDF91CF9101
:106840001F9108950895CF93809187048823A1F024
:10685000C091E900CF709091EC00892F817090FD7C
:1068600080E8C82B1092E9008091E80083FD0E9427
:10687000D032CF70C093E900CF910895AA1BBB1B03
:1068800051E107C0AA1FBB1FA617B70710F0A61B30
:10689000B70B881F991F5A95A9F780959095BC0151
:1068A000CD01089597FB072E16F4009407D077FDCD
:1068B00009D00E943E3407FC05D03EF490958195A6
:1068C0009F4F0895709561957F4F0895EE0FFF1FBC
:1068D0000590F491E02D0994692796276927782778
:1068E000872778270895FB01DC0102C005900D92EF
:1068F00041505040D8F70895FB01DC0102C00190DF
:106900000D9241505040D8F70895DC0101C06D93BD
:1069100041505040E0F70895DC01CB01FC01F999AA
:10692000FECF06C0F2BDE1BDF89A319600B40D92DB
:1069300041505040B8F70895F999FECF92BD81BDFE
:10694000F89A992780B50895A8E1B0E042E050E0B8
:106950000C948E34262FF999FECF92BD81BDF89A02
:10696000019700B4021639F01FBA20BD0FB6F89493
:10697000FA9AF99A0FBE08950396272F0E94AB3416
:106980000E94AA34252F0E94AB34242F0C94AB34E0
:106990000196272F0E94AB340C94AA34DC01CB0162
:1069A00003C02D910E94D93441505040D0F7089532
:1069B000262FF999FECF1FBA92BD81BD20BD0FB61B
:1069C000F894FA9AF99A0FBE01960895F894FFCFB9
:1069D000650865086E086E0870086E086E086E0817
:1069E0006508650875086E086E087508BA08BA0863
:1069F0001D091D099D09B709EA08EA08C4092D0AFD
:106A00003E0A3E0ACE0AEA08EA08D70A4B1D7B1D59
:106A1000831D6D1D6D1DBE1DCD1DDC1D6D1DE71D76
:106A2000F01DFD1D081E0B1EF93221330A342133DF
:0C6A30000A34543375330A34CC33D833A5
:106A3C0010022808641E140A321E0100010800FF0F
:106A4C0001AF00F82C4E2D2D2D292D252D012E6357
:106A5C00E0AAFBE4953090919293959497F7F6F514
:106A6C003136353496E200E900EA00B500B600B7DD
:106A7C0000CD008301CC008A0192019401210223F4
:106A8C000224022502260227022A02B300B4006F58
:106A9C00007000818283E200E900EA00B500B600D4
:106AAC00B700CD008301CC008A0192019401210230
:106ABC00230224022502260227022A02B300B40074
:106ACC006F0070008182834022BC0B062D054F05A0
:066ADC00D204EB040B05DF
:00000001FF
